:100000000C94702D0C94212E0C94212E0C94212EE6
:100010000C94212E0C94212E0C94212E0C94212E24
:100020000C94212E0C94212E0C94212E0C94212E14
:100030000C94212E0C94D9410C94212E0C94212E39
:100040000C94212E0C94212E0C94212E0C94212EF4
:100050000C94212E0C94212E0C94212E0C94212EE4
:100060000C94212E0C94212E0C94212E0C94212ED4
:10007000040004002700280029002A002B002C007F
:100080002D002E002F0030003000310032003300F0
:1000900034003500000000000000000000000000F7
:1000A0000000000000000000000000000000000050
:1000B0000000000000000000000000000000000040
:1000C0000000000000000000000000000000000030
:1000D0000000000000000000000000000000000020
:1000E00000000000000000490000004952520000DA
:1000F00052525C2D000000000000000000000000D3
:10010000000000000040000000494A5200495252DD
:100110005B1C52531C25241B2425251B0A0A2D1C5D
:1001200012120A0A0000000000000000404949497C
:100130004949525B5B5B525B1C1C1312241C120965
:10014000090912090909090A0A0A0A0A0A13120AFC
:100150000A12130A0000000000009252525252523A
:1001600013121309001C0A1212401B65090A000928
:10017000241B120000251C1C010025241C1C00242B
:1001800025242424000000000000524949400000BA
:100190001B1352494900641C1C5B4A481C651C2502
:1001A00052491C1C652464491C1C652564491C1C9F
:1001B0006D2E5C49000000000000000000000049B6
:1001C00000000000535200000053522500004A5224
:1001D000252500005B251300005B53000A1C095B0A
:1001E0001C657F374052522E2E1C525C2E251B134D
:1001F00024251C1C12002525120000121B000013D0
:100200002E37001B37372E2E37372E2E2E2E2E2E22
:100210006E6E6E1C131312000913120000121313DA
:100220000012251C13132E371C131313361C131B1B
:100230001B1B25131C1C1B1B1B1C1C1C1C1C1C1C03
:100240001C1C1C131312121313001313131C00098C
:1002500013131C010037131C13002E2E1C1C001C32
:10026000772E2500137F251C010A37241C1C0A2E1B
:1002700025250900132E242525252E252525252570
:1002800025252D2E251B2E2E251C1325251C1C1C3B
:100290001C011C1C1300011C0A000165775C016E27
:1002A0007F6E521B25256D1C524925251C135300BA
:1002B0001C1C1C524A001B135B5B000009525C00B3
:1002C00000005B5C000000001B000000000000005C
:1002D00000000000135B7F776E6E136577766E6E9D
:1002E0001B65777676761B5BBF76B67609136DBF96
:1002F000B7B6001B125C76BF0000121B125B000039
:100300000000090A6E6E6E77241C6E6E77251C1C29
:100310006E776E1C1C1C76761C1C2425B765646DDC
:100320006D1B766D6D5B09125B5C5B125B64121377
:10033000131B12121C1C1C1C1C241C1C24252524F1
:100340002425251B00002513000064BF00096EBF93
:10035000BF6D6EBF6D5B12135B12131209000901B2
:10036000000000002E1C0900096E010009767F7F45
:1003700012777F7F6412BF775B121B095B121B0928
:1003800000001B0900000000000000000000000049
:10039000000000007F7F5313130064121B01000054
:1003A0001B12000000000000000000000000000020
:1003B000000000000000000000000000000000003D
:1003C00000000000000000000000260000002600E1
:1003D0002F0000002F00370000003700FF00000052
:1003E000FF00BF000000BF003700003700000026FC
:1003F0002600000000000000000026262626260019
:10040000000000002F000000003700000000FF0087
:10041000000000BF0000000037000000000026269A
:10042000262626000000000000002626262626009C
:100430002F0000000000370000000000FFFFFFFF5A
:100440000000BF000000000037000000000026266A
:100450002626260000000000000026262626000092
:100460002F0000002F00370000003700FFFFFFFFC4
:100470000000BF000000BF00370000003700262644
:1004800026260000000000000000000026262600AE
:10049000002F00002F00370000003700FF00000091
:1004A000FF00BF000000BF00370000370000262615
:1004B00026000000000000000000260000002600CA
:1004C0002F0000002F000037003700000000FF0061
:1004D000000000BF00BF000037000000370026000A
:1004E00000002600000000000000000000000000E6
:1004F00000000000000000000000000000000000FC
:10050000000000000000009B000000529BA40000BF
:100510005B9B6D7700000000000000000000000001
:1005200000000000005B000000E4F6FF099BEDF610
:10053000FFBFA4ADBFBFBFBF767F7FB7B7BF7F761A
:100540006EB7B7BF00000000000000005BB6F6F613
:10055000F6FFFFFFFFBFFFFFFFBFBFAEFFFFFFB70D
:10056000AD65FFFFB7B6AD65FFFFBFB7AE6EFFFF6E
:10057000BFB7B765000000000000F6F6EDEDADA4D2
:10058000B66D6D5C526E6565655265765C5C525306
:100590006E246552526E25255B52772D2525526EAD
:1005A0006E2D2525000000000000A49B9B49000043
:1005B0006564A49B92006D2525649349656E652E44
:1005C0009B5224256D25655225246D2D65522525C8
:1005D0006E2E645200000000000000000000004A7F
:1005E000000000005B9B0000005B5B2D0000525B85
:1005F0002E2E00015B2D1C01005C5B014A654A5BED
:100600001C6E7F77495B9B77776D5B65776E656561
:100610006D2D25255C522E25130949641C09095CA2
:100620007F7F091C7F7F777F777F77777F7F7776E4
:10063000777F7F6E656E6EA4B6FF655BA4B7BFFF64
:10064000526DBFBFBFFF7FBFBFBFBFFFBFBFB7BF41
:10065000FFFF7FB7BFBFFFFF6EB7BFBFFFFF77BF13
:10066000BFBFFFFFFFFFBFBFB75BFFFFBFBFA464FC
:10067000FFFFBFADA47FFFFFBFA4BF7FFFBFADBF24
:10068000BFBFFFB6BFBFBF77F7BFBFBF7777FFBFA3
:10069000BFBF64526D7F6E2E2D2D7F766E6E6E2ED7
:1006A000777777762E1C7F776E251C257765252535
:1006B0001C096E6E1C0949255B494A6E7F6453779D
:1006C000BF775B5C256E6E255B4A25651C1B5B0056
:1006D0002524245B53001C1B5B5C00000A5B640048
:1006E00000006464000000005C00000000000000E6
:1006F000000000005B5C7FBF77765C6D7FB777772B
:100700005C6D7FBF77775C64BFBFBFBF0A5C6EBFA5
:10071000BFBF0065646DBFBF00005B6D646D00000E
:100720000000125B7777777F6E6E77777F766D76D6
:1007300077BF776D6E76BF7F6D6E767FBF7676BF43
:10074000BF76BFBFBFB664ADADB6B6ADBFFF646D1B
:10075000ADB6AD6477BFBFBFFFFF77BFBFBFFFFFC1
:100760007FBFBFBFFFF6BFB7ADF6FFFFA4ADFFFF72
:10077000FFFFFFFFFFFFFFFFFFFFFFF6A4005B523D
:1007800000000000BFBFAD5B64BFB6ADADBFFFBF33
:10079000FFFFFFFFBF64FFFFBFB6765BFFBFBF5B1E
:1007A0000000FF5C000000000000000000000000EE
:1007B00000000000BFBF645C5C006E5C6549000027
:1007C0006D5B000000000000000000000000000061
:1007D0000000000000000000000000000000000019
:1007E0000000000000000000000000000000000009
:1007F0000000000000000000000000FF00000000FA
:10080000FFFF000000FFFFFF000000FFFFFF0000F0
:1008100000FFFFFF000000FFFFFF00FFFFFFFFFFE3
:10082000FFFFFFFFFFFFFFFFFFFFFFFFFFFFFFFFD8
:10083000FFFFFFFFFFFFFFFFFFFFFFFFFFFFFFFFC8
:10084000FFFFFFFFFFFFFF000000FFFFFFFFFF00B4
:10085000FFFFFFFFFFFFFFFFFFFFFFFFFFFFFFFFA8
:10086000FFFFFFFFFFFFFFFFFFFFFFFFFFFFFFFF98
:10087000FFFFFFFF0000000000000000000000007C
:10088000000000000000FF0000000000FFFF00006B
:100890000000FFFFFF000000FFFFFF000000FFFF60
:1008A000FF000000000000FFFFFF000000FFFFFF4F
:1008B000000000FFFFFF00000000FFFF000000003D
:1008C00000FF000000000000000000000000000029
:1008D00000000000FFFFFFFFFFFFFFFFFFFFFFFF24
:1008E000FFFFFFFFFFFFFFFFFFFFFFFFFFFFFFFF18
:1008F000FFFFFFFFFFFFFFFF00FFFFFFFFFF000005
:10090000FFFFFFFFFFFFFFFFFFFFFFFFFFFFFFFFF7
:10091000FFFFFFFFFFFFFFFFFFFFFFFFFFFFFFFFE7
:10092000FFFFFFFFFFFFFFFFFFFFFFFFFF00FFFFD6
:10093000FFFF0000FFFFFF000000FFFFFF000000BF
:10094000FFFFFF000000FFFF00000000FF000000AD
:100950000000000000000000000000000000000097
:10096000000000004242424242424242424242426F
:100970004242420442424242420442424242420411
:1009800042424242420442424242420442424242C3
:100990004204424242424242424242424242424275
:1009A0004242424242424242424242424242424227
:1009B0004242424242424242424242424242424217
:1009C0004242424242424242424242424242424207
:1009D00042420442424242420442424242420442B1
:1009E0004242424204424242424204424242424263
:1009F000044242420000000080800000000080802D
:100A000000000000808000000000808000000000E6
:100A100080800000000080800000000080800000D6
:100A200000008080808080808080808080808080C6
:100A300080808080808080808080808080800000B6
:100A400000008080000000008080000000008080A6
:100A50000000000080808080808080808080808096
:100A60008080808080808080808080800000000086
:100A70008080000000008080000000008080000076
:100A80000000808080800000000080800000000066
:100A90008080000000008080000000008080000056
:100AA0000000808000000000808000000000808046
:100AB00000000000C7C7C7C7C7C7C7C7C7C7C7C7E2
:100AC000C7C7C7C7C7C7C7C7C7C7C7C7C7C7C7C7B6
:100AD000C7C7C7C7C7C7C7C7C7C7C7C7C7C7C7C7A6
:100AE000C7C7C7C7060004000000010002000300DA
:100AF0000400050006000700080009000A000B00BA
:100B00000C000D000E000F0010000000110012007C
:100B10001300140015001600060003000000170063
:100B2000180019001A001B001C001D001E001F00E9
:100B300020002100220023002400250026000000C0
:100B400000020800085504085A0000F80009900047
:100B50000A1E32050000FF000000400B00000000EC
:100B60000E2F1C2FE72F943380331F2F2E2F3D2F56
:100B700068334B2F592F00000001000200030004CE
:100B80000005010001010102010301040105020049
:100B90000201020202030204020503000301030230
:100BA0000303030403050400040104020403040412
:100BB00004050500050105020503050405050600F9
:100BC00006010602060306040605070007010702E0
:100BD00007030704070508000801080208030804C2
:100BE00008050900090109020903090409050A00A9
:100BF0000A010A020A030A040A050B000B010B0290
:100C00000B030B040B050C000C010C020C030C0471
:100C10000C050D000D010D020D030D040D050E0058
:100C20000E010E020E030E040E050F000F010F023F
:100C30000F030F040F051000100110021003100421
:100C40001005110011011102110311041105120008
:100C500012011202120312041205130013011302EF
:100C600013031304130514001401140214031404D1
:100C700014051500150115021503150415051600B8
:100C8000160116021603160416051700170117029F
:100C90001703170417051800180118021803180481
:100CA00018051900190119021903190419051A0068
:100CB0001A011A021A031A041A051B001B011B024F
:100CC0001B031B041B051C001C011C021C031C0431
:100CD0001C051D001D011D021D031D041D051E0018
:100CE0001E011E021E031E041E051F001F011F02FF
:100CF0001F031F041F05000000000000000000008B
:100D000000000000000000000000000000000000E3
:100D100000000000000000000000000000000000D3
:100D2000000000000000E8E8E8E8E8E8E8D8D8D8E3
:100D3000D880E8D8D8D8D880E8D8D8D8D880E8D80B
:100D4000D8D8D880E8D8D8D8D880E8D8D8D8D8800B
:100D5000E88080808080808080D8D8D8808080D8CB
:100D6000D8D8808080D8D8D8808080D8D8D8D8D813
:100D7000D8808080D8D8D8808080D8D8D88080800B
:100D8000D8D8D8808080808080D8D8D88080E8E883
:100D9000D8D88080E8E8D8D880E8E8E8E8D8D8E86B
:100DA000E8E8E880D8D8E8E88080D8D8E8E880800B
:100DB000D8D8D880808042424242424242858585CE
:100DC00085424285CDCD85424285CDCD8542428545
:100DD000CDCD85424285CDCD8542428585858542F2
:100DE000424242424242424242424242428585851A
:100DF00085424285CDCD85424285CDCD8542428515
:100E0000CDCD85424285CDCD8542428585858542C1
:100E1000424242424242FEFEFFFFFEFEFEFFFFFF55
:100E2000FFFEFEFFFFFFFFFEFEFEFFFFFEFE424253
:100E300042424242424242424242FF00000000FF20
:100E4000FE00FEFE00FE00000000000000000000AA
:100E50000000000000000000000000000000000092
:100E60000000000000000000000000000000000082
:100E70000000000000000000FF00000000FFFFFF76
:100E8000000000FFFFFF00000000FF000000000066
:100E9000FF0000000000000000000000FF00000054
:100EA000000000000000FFFF00FFFF00FFFF00FF49
:100EB000FF00FF0000FF0000000000000000000035
:100EC0000000000000000000000000000000000022
:100ED00000000000000000000000000000FF00FF14
:100EE0000000FFFFFFFFFF0000FF00FF000000FF0A
:100EF00000FF0000FFFFFFFFFF0000FF00FF0000FA
:100F000000000000000000FF0000000000FFFFFFE5
:100F10000000FF000000000000FFFF0000000000D4
:100F200000FF0000FFFFFF0000000000FF000000C6
:100F3000000000000000FFFF0000FF00FFFF0000B6
:100F4000FF00000000FF00000000FF00000000FFA5
:100F500000000000FF0000FFFF00FF0000FFFF0097
:100F600000000000000000FF00000000FF00FF0084
:100F70000000FF00FF00000000FF00000000FF0075
:100F8000FF00FF00FF0000FF000000FFFF00FF0068
:100F900000000000000000FFFF00000000FFFF0055
:100FA000000000FF00000000000000000000000042
:100FB0000000000000000000000000000000000031
:100FC0000000000000000000FF00000000FF000023
:100FD000000000FF0000000000FF0000000000FF14
:100FE0000000000000FF000000000000FF00000003
:100FF00000000000000000FF000000000000FF00F3
:1010000000000000FF0000000000FF0000000000E2
:10101000FF0000000000FF00000000FF00000000D3
:1010200000000000000000000000000000FF00FFC2
:10103000000000FFFFFF0000FFFFFFFFFF0000FFB9
:10104000FFFF000000FF00FF0000000000000000A4
:101050000000000000000000000000000000FF0091
:1010600000000000FF000000FFFFFFFFFF00000086
:10107000FF0000000000FF00000000000000000072
:101080000000000000000000000000000000000060
:101090000000000000000000000000000000000050
:1010A0000000000000FFFF00000000FFFF00000044
:1010B00000FF000000000000000000000000000031
:1010C0000000000000000000FFFFFFFFFF00000025
:1010D0000000000000000000000000000000000010
:1010E0000000000000000000000000000000000000
:1010F00000000000000000000000000000000000F0
:101100000000000000FFFF00000000FFFF000000E3
:1011100000000000000000000000000000000000CF
:10112000FF00000000FF00000000FF00000000FFC3
:1011300000000000FF0000000000000000000000B0
:1011400000000000000000373737000037000000C3
:1011500037003700003737003700370037003737A0
:101160000000370037000000370000373737000035
:1011700000000000000000003700000000373700CA
:1011800000000000370000000000370000000000F1
:10119000370000000000370000000037373700003C
:1011A0000000000000000037373700003700000063
:1011B000370000000000370000003737000000371C
:1011C00000000000370000000000373737373700D5
:1011D0000000000000000037373700003700000033
:1011E00037000000000037000037373700000000EC
:1011F00000003700370000003700003737370000A5
:101200000000000000000000003700000000373739
:101210000000003700370000370000370000373784
:1012200037373700000000370000000000370000AB
:101230000000000000003737373737003700000064
:10124000000037000000000037373737000000008B
:101250000000370037000000370000373737000044
:1012600000000000000000003737000000370000D9
:101270000000370000000000373737370000370024
:101280000000370037000000370000373737000014
:10129000000000000000373737373700000000003B
:1012A0003700000000370000000037000000003762
:1012B00000000000003700000000003700000000C0
:1012C0000000000000000037373700003700000042
:1012D000370037000000370000373737000037008D
:1012E00000003700370000003700003737370000B4
:1012F0000000000000000037373700003700000012
:10130000370037000000370000373737370000005C
:1013100000003700000000370000003737000000F1
:1013200000000000000000000000000000000000BD
:10133000000000FFFF00000000FFFF0000000000B1
:101340000000000000FFFF00000000FFFF000000A1
:10135000000000000000000000000000000000008D
:10136000000000FFFF00000000FFFF000000000081
:101370000000000000FFFF00000000FFFF00000071
:1013800000FF0000000000000000FF00000000FF60
:1013900000000000FF00000000FF0000000000004F
:1013A000FF000000000000FF000000000000FF0040
:1013B000000000000000000000000000000000002D
:1013C0000000FFFFFFFFFF00000000000000000022
:1013D00000000000FFFFFFFFFF0000000000000012
:1013E00000000000000000FF000000000000FF00FF
:1013F0000000000000FF000000000000FF000000EF
:1014000000FF00000000FF00000000FF00000000DF
:1014100000000000000000FFFFFF0000FF000000D0
:10142000FF0000000000FF000000FFFF00000000C0
:10143000FF0000000000000000000000FF000000AE
:1014400000000000000000FFFFFF0000FF000000A0
:10145000FF00FF00FFFFFF00FF00FF00FF00FF0095
:10146000FFFFFF00FF000000000000FFFFFF000083
:1014700000000000000000FFFFFF0000FF00000070
:10148000FF00FF000000FF00FF000000FF00FFFF63
:10149000FFFFFF00FF000000FF00FF000000FF0053
:1014A000000000000000FFFFFFFF0000FF00000041
:1014B000FF00FF000000FF00FFFFFFFF0000FF0034
:1014C0000000FF00FF000000FF00FFFFFFFF000023
:1014D00000000000000000FFFFFF0000FF00000010
:1014E000FF00FF0000000000FF0000000000FF0000
:1014F00000000000FF000000FF0000FFFFFF0000F1
:10150000000000000000FFFFFFFF0000FF000000E0
:10151000FF00FF000000FF00FF000000FF00FF00D1
:101520000000FF00FF000000FF00FFFFFFFF0000C2
:10153000000000000000FFFFFFFFFF00FF000000B1
:101540000000FF0000000000FFFFFFFF0000FF00A1
:1015500000000000FF0000000000FFFFFFFFFF0091
:10156000000000000000FFFFFFFFFF00FF00000081
:101570000000FF0000000000FFFFFFFF0000FF0071
:1015800000000000FF0000000000FF00000000005D
:1015900000000000000000FFFFFF0000FF0000004F
:1015A000FF00FF0000000000FF00FFFFFF00FF0042
:1015B0000000FF00FF000000FF0000FFFFFFFF0032
:1015C000000000000000FF000000FF00FF0000001E
:1015D000FF00FF000000FF00FFFFFFFFFF00FF0014
:1015E0000000FF00FF000000FF00FF000000FF0000
:1015F00000000000000000FFFFFF00000000FF00EF
:1016000000000000FF0000000000FF0000000000DC
:10161000FF0000000000FF00000000FFFFFF0000CF
:1016200000000000000000000000FF0000000000BB
:10163000FF0000000000FF0000000000FF00FF00AE
:101640000000FF00FF000000FF0000FFFFFF0000A0
:10165000000000000000FF000000FF00FF0000FF8E
:101660000000FF00FF000000FFFF00000000FF007F
:10167000FF000000FF0000FF0000FF000000FF006F
:10168000000000000000FF0000000000FF0000005C
:101690000000FF0000000000FF0000000000FF004D
:1016A00000000000FF0000000000FFFFFFFFFF0040
:1016B000000000000000FF000000FF00FFFF00FF2F
:1016C000FF00FF00FF00FF00FF000000FF00FF0021
:1016D0000000FF00FF000000FF00FF000000FF000F
:1016E000000000000000FF000000FF00FFFF0000FE
:1016F000FF00FF00FF00FF00FF0000FFFF00FF00F2
:101700000000FF00FF000000FF00FF000000FF00DE
:1017100000000000000000FFFFFF0000FF000000CD
:10172000FF00FF000000FF00FF000000FF00FF00BF
:101730000000FF00FF000000FF0000FFFFFF0000AF
:10174000000000000000FFFFFFFF0000FF0000009E
:10175000FF00FF000000FF00FFFFFFFF0000FF0091
:1017600000000000FF0000000000FF00000000007B
:1017700000000000000000FFFFFF0000FF0000006D
:10178000FF00FF000000FF00FF000000FF00FF005F
:10179000FF00FF00FF0000FF000000FFFF00FF0050
:1017A000000000000000FFFFFFFF0000FF0000003E
:1017B000FF00FF000000FF00FFFFFFFF0000FF0031
:1017C00000FF0000FF000000FF00FF000000FF001E
:1017D00000000000000000FFFFFF0000FF0000000D
:1017E000FF00FF000000000000FFFFFF00000000FE
:1017F0000000FF00FF000000FF0000FFFFFF0000EF
:10180000000000000000FFFFFFFFFF000000FF00DE
:1018100000000000FF0000000000FF0000000000CA
:10182000FF0000000000FF0000000000FF000000BB
:10183000000000000000FF000000FF00FF000000AB
:10184000FF00FF000000FF00FF000000FF00FF009E
:101850000000FF00FF000000FF0000FFFFFF00008E
:10186000000000000000FF000000FF00FF0000007B
:10187000FF00FF000000FF00FF000000FF00FF006E
:101880000000FF0000FF00FF00000000FF0000005C
:10189000000000000000FF000000FF00FF0000004B
:1018A000FF00FF00FF00FF00FF00FF00FF00FF0040
:1018B000FF00FF00FF00FF00FF0000FF00FF00002F
:1018C000000000000000FF000000FF00FF0000001B
:1018D000FF0000FF00FF00000000FF00000000FF0D
:1018E00000FF0000FF000000FF00FF000000FF00FD
:1018F000000000000000FF000000FF00FF000000EB
:10190000FF00FF000000FF0000FF00FF00000000DC
:10191000FF0000000000FF0000000000FF000000CA
:10192000000000000000FFFFFFFF0000000000FFBC
:1019300000000000FF00000000FF00000000FF00AA
:1019400000000000FF0000000000FFFFFFFF00009C
:101950000000000000000000FFFF000000FF00008A
:10196000000000FF00000000FFFF0000000000FF7B
:101970000000000000FF000000000000FFFF00006A
:101980000000000000000000FFFF000000FF00005A
:10199000FF00FF00FFFF00FFFF00FF0000FFFF0050
:1019A000FFFF00FF00FF0000FF000000FFFF00003E
:1019B00000000000000000FFFF000000000000FF2A
:1019C0000000000000FF0000000000FFFF0000001A
:1019D00000FF0000000000FF000000FFFF0000000B
:1019E000000000000000C7C7C7C7C7C7C7C7C7C731
:1019F000C7C7C7C7C7C7C7C7C7C7C7C7C7C7C7C777
:101A0000C7C7C7C7C7C7C7C7C7C7C7C7C7C7C7C766
:101A1000C7C7C7C7C7C752520909090900520909F0
:101A2000090900000909520900000052520900008A
:101A30000000520900000000000000000000000942
:101A400000000000000009520909091109090909EB
:101A50000952095252520909095209090909005249
:101A6000525109090052520909090052090000099E
:101A700009525209095252520900095252520900A0
:101A800009090909090952090909090009095252F4
:101A900052005209090909095209520900000909AD
:101AA0005209095252000900090952520900090954
:101AB00009090900520900520900090909520909D6
:101AC00052520909090952525252090909095B5235
:101AD000000909520052525209090009090909096D
:101AE00000095200095200095209090900090909AF
:101AF00052520909525252520909525B0909090905
:101B000052005209090052090009525209090009FC
:101B1000525209520909090909090009090909521A
:101B200000525252095209090909090900000952D3
:101B300000525209095211090909520952090909A9
:101B400009090909525252090909090952090909E1
:101B5000515252000909095252000900000952006D
:101B60005209095252090909090952520909090978
:101B7000520009520909000009525200000009529E
:101B8000000000000000000000000900000000004C
:101B90000000000000000000000000000000000045
:101BA0000000000000000000000000000000000035
:101BB0000000000000000000000000000000000025
:101BC0000000000000000000000000000000000015
:101BD0000000000000000000000000000000000005
:101BE00000000000000000000000000000000000F5
:101BF00000000000000000000000000000000000E5
:101C000000000000000000000000000000000000D4
:101C100000000000000000000000000000000000C4
:101C200000000000000000000000000000000000B4
:101C30000052000000000952000000525252000001
:101C400000090909000009090000000909520900FA
:101C500009000952090900000000000052000000BC
:101C60000000520900000000525252000000090911
:101C700009000000000009090000000952090900DC
:101C800009095209000900000000000000000000DE
:101C90000000000000000000000000000000000044
:101CA0000000000000000000000000000000000034
:101CB0000000000000000000000000000000000024
:101CC0000000000000000000000000000000000014
:101CD0000000000000000000000000000000000004
:101CE00000000000000000000000000000000000F4
:101CF00000000000000000000000000000000000E4
:101D000000000000000000000000000000000000D3
:101D100000000000000000000000000000000000C3
:101D200000000000000000000000000000000000B3
:101D300000000000000000000000000000000000A3
:101D40000000000000000052520909520000520930
:101D5000095200005209525200000009090900000E
:101D6000000052090000000052090000000000526B
:101D7000000000000000525252520909520909099C
:101D800009090909000000000909090909000909F0
:101D900052090909090952090909090952090909D8
:101DA00009005209000909525209005252525209BF
:101DB0000952000909090952095252520952525254
:101DC00052525252525209090909090909090909CD
:101DD000090909090909520009525209520909520F
:101DE00052525209090909005209525252095252DB
:101DF000525252520909090952520909090909099D
:101E0000090909090909090952525252090909091E
:101E10000952000000000909000909090909090916
:101E20000952090909090952090909090952090947
:101E30000900095200095209095252005209095277
:101E4000000052520952000009090900000009521D
:101E500000000000095200000000520000000000D5
:101E60000000000000000000000000000000000072
:101E70000000000000000000000000000000000062
:101E80000000000000000000000000000000000052
:101E90000000000000000000000000000000000042
:101EA0000000000000000000000000000000000032
:101EB0000000000000000000000000000000000022
:101EC0000000000000000000000000000000000012
:101ED0000000000000000000000000000000000002
:101EE00000000000000000000000000000000000F2
:101EF00000000000000000000000000000000000E2
:101F0000000900000000525B000000005252000077
:101F10000009090900005209525200095209095BDF
:101F200000095200005209000909090909090909B3
:101F300000525209090909095209090909520909F6
:101F40005209525209095209095209090909090994
:101F50005252520952090909090900095200090996
:101F60000909090909090952520909090952525274
:101F700009520909520909520909090909090909F6
:101F800009520952525200000000000009000000EE
:101F900000005B52000000005252000000000909DE
:101FA000090000005252095200005B090952090061
:101FB0005200005209000000000000000000000074
:101FC0000000000000000000000000000000000011
:101FD0000000000000000000000000000000000001
:101FE00000000000000000000000000000000000F1
:101FF00000000000000000000000000000000000E1
:1020000000000000000000000000000000000000D0
:1020100000000000000000000000000000000000C0
:1020200000000000000000000000000000000000B0
:1020300000000000000000000000000000000000A0
:102040000000000000000000000000000000000090
:102050000000000000000000000000000000000080
:102060000000000000000000000000000000000070
:10207000000000000000000952000052000952094F
:10208000095B0000520952520000000909090000D2
:102090000000525200000000525B000000000009E6
:1020A00000000000000052525209520909090909B2
:1020B00009090909520909520909520952525209DA
:1020C00009090952520909090909090909090052AE
:1020D0000900090909090952095252520909090955
:1020E00009095209095209095252095209095209AA
:1020F000090909520909090909525200090909097E
:102100000909090900095200005209005B09095236
:1021100009005252095200000909090000005252F8
:10212000000000005B5200000000090000000000F9
:10213000000000000000000000000000000000009F
:10214000000000000000000000000000000000008F
:10215000000000000000000000000000000000007F
:10216000000000000000000000000000000000006F
:10217000000000000000000000000000000000005F
:10218000000000000000000000000000000000004F
:10219000000000000000000000000000000000003F
:1021A000000000000000000000000000000000002F
:1021B000000000000000000000000000000000001F
:1021C000000000000000000000000000000000000F
:1021D00000520000000052090000000052090000F7
:1021E000000909090000520952520000520909521F
:1021F00000525209095209005209000909095209FD
:1022000009090909520909090909520909090909AC
:102210000909090009090000000052090909090912
:1022200052525252090909090909090909090909FA
:10223000090952520909090952525252525209527D
:1022400052520952000909090952525252090952BF
:10225000095252090052090909090909090909091C
:10226000090909090909525252525252525252094D
:10227000525252095209090909005209095252528F
:10228000520009525209090009520009090909526C
:102290000909090909520909090909520909000925
:1022A0000909090900000000090909090909095279
:1022B0000909525252520000000000005200000072
:1022C0000000095200000000095200000000090946
:1022D0000900000052520952000052090952000040
:1022E00052090952520000000000000000000000E6
:1022F00000000000000000000000000000000000DE
:1023000000000000000000000000000000000000CD
:1023100000000000000000000000000000000000BD
:1023200000000000000000000000000000000000AD
:10233000000000000000000000000000000000009D
:10234000000000000000000000000000000000008D
:10235000000000000000000000000000000000007D
:10236000000000000000000000000000000000006D
:10237000000000000000000000000000000000005D
:10238000000000000000000000000000000000004D
:10239000000000000000000000000000000000003D
:1023A0000000000000000900095209090009095253
:1023B00009000000090900000000000909090000E7
:1023C000005252520000000009520000000000526A
:1023D0000000000000000909520900090009520923
:1023E0000900000009090000090909000000525213
:1023F00052000000520900000000520000000000DE
:1024000000000000000000000000000000000000CC
:1024100000000000000000000000000000000000BC
:1024200000000000000000000000000000000000AC
:10243000000000000000000000000000000000009C
:10244000000000000000000000000000000000008C
:10245000000000000000000000000000000000007C
:10246000000000000000000000000000000000006C
:10247000000000000000000000000000000000005C
:10248000000000000000000000000000000000004C
:10249000000000000000000000000000000000003C
:1024A00000090000000000000000000052090000C8
:1024B000005252090000090952090052090909098C
:1024C00052520909090909525209095200520900D8
:1024D00000090052520909090052525109090952D2
:1024E0000909090909525252090909090909095238
:1024F00009520909091152090952520052090000F2
:1025000009090909090952095252520052090909D7
:102510000900090909090909520952520900090962
:1025200052520900095200090952005209090909C9
:102530005B520909525252520909525209090900C3
:10254000090909520900520900520900090909093B
:10255000090009095252520052090900525B090947
:1025600009095252525209090909525209095209DC
:10257000090900095200095200090909090900095D
:102580005252090900090052520909520909000072
:1025900009520952090909090952005252520909FE
:1025A00000090909095209090909090900095252D2
:1025B00052090009525252090952520909000009F0
:1025C00052000909095252000909515252000909E1
:1025D00009095209090952525209520909090909FE
:1025E000110909095209000000000000090000005B
:1025F0000000000000000000095200000000095225
:102600005200000009520909000009090909520095
:10261000090909095252C7C7C7C7C7C7C7C7C7C72C
:10262000C7C7C7C7C7C7C7C7C7C7C7C7C7C7C7C73A
:10263000C7C7C7C7C7C7C7C7C7C7C7C7C7C7C7C72A
:10264000C7C7C7C7C7C70000E2E2E2E200E2E2E2B2
:10265000E2E200E2E2E2E2E200E2E2E2E2E2E2E21E
:10266000E2E2E2E2E2E2E2E2E2E2E2E2E2E2E2E24A
:10267000E2E2E2E2E2E2E2E2E2E2E200E2E2E2E21C
:10268000E2E2E2E2E2E2E2E2E2E2E2E2E2E2E2E22A
:10269000E2E2E2E2E2E2E2E2E2E2E2E2E2E2E2E21A
:1026A000E2E2E2E2E20000000000000000000000C0
:1026B0000000E20000000000E20000000000E20074
:1026C00000000000E2000000000000000000000028
:1026D00000000000000000000000000000000000FA
:1026E00000000000000000000000000000000000EA
:1026F00000000000000000000000000000000000DA
:102700000000000000000000000000E200000000E7
:10271000E2E200000000E2E200000000E2E200006D
:102720000000E2E200000000E2E200000000E2E25D
:1027300000000000E2E2E20000000000E200000011
:102740000000E20000000000E2E200000000E2E21F
:1027500000000000E2E200000000E2E200000000F1
:10276000E2E20000000000E2E200000000E2E2E23B
:10277000000000E2E2E20000E2E2E2E20000E2E267
:10278000E2E20000E2E2E2E20000E2E2E2E2000075
:10279000E2E2E2E2000000000000E2E2000000E20B
:1027A000E2E20000E2E2E2E20000E2E2E2E2000055
:1027B000E2E2E2E20000E2E2E2E20000E2E2E2E281
:1027C0000000E2E2E2E2E2E2E2E2E2E2E2E2E2E2AD
:1027D000E2E2E2E2E2E2E2E2E2E2E2E2E2E2E2E2D9
:1027E000E2E2E2E2E2E2E2E2E2E2E2E2E2E2E2E2C9
:1027F000E2E2E2E2E2E2000000000000E2000000AB
:102800000000E2E200000000E2E200000000E2E27C
:1028100000000000E2E200000000E2E20000000030
:10282000E2E20000000000000000000000000000E4
:102830000000000000000000000000000000000098
:10284000000000E20000000000E20000000000E2E2
:102850000000000000E200E2E2E2E2E2E2E2E2E2A4
:10286000E2E2E2E2E2E2E2E2E2E2E2E2E2E2E2E248
:10287000E2E2E2E2E2E2E2E2E2E2E2E2E2E2E2E238
:10288000E2E2E2E2E2E2E2E2E2E20000E2E2E2E2EC
:10289000E200E2E2E2E2E200E2E2E2E2E200E2E2BE
:1028A000E2E2E2E2E2E2E2E2E2E2E2E2E2E2E2E208
:1028B000E2E2E2E2E2E2E2E2E2E20000E2E2E2E2BC
:1028C0000000E2E2E2E20000E2E2E2E20000E2E234
:1028D000E2E20000E2E2E2E20000E2E2E2E2000024
:1028E000E2E2E2E2000000000000E2E2000000009C
:1028F000E2E200000000E2E200000000E2E200008C
:102900000000E2E200000000E2E200000000E2E27B
:1029100000000000E2E2E2E200000000E2E200006B
:102920000000E2E200000000E2E200000000E2E25B
:1029300000000000E2E200000000E2E2000000000F
:10294000E2E2000000000000E2E2E2E20000E2E277
:10295000E2E20000E2E2E2E20000E2E2E2E20000A3
:10296000E2E2E2E20000E2E2E2E20000E2E2E2E2CF
:102970000000E2E2E2E20000000000E200000000ED
:1029800000E20000000000E20000000000E20000A1
:10299000000000E20000000000E20000000000E291
:1029A0000000000000E2E2E2E2E2E2E2E2E2E2E271
:1029B000E2E2E2E2E2E2E2E2E2E2E2E2E2E200E2D9
:1029C000E2E2E2E200E2E2E2E2E200E2E2E2E2E2AB
:1029D0000000E2E2E2E2E2E2E2E2E200E2E2E2E27D
:1029E000E2E2E2E2E2E2E2E2E2E2E2E2E2E2E2E2C7
:1029F000E2E2E2E2E2E2E2E2E2E2E2E2E2E2E2E2B7
:102A0000E2E2E2E2E2E2000000000000000000007A
:102A100000000000000000E20000000000E2E20010
:102A2000000000E2E200000000E2E200000000E23C
:102A3000E200000000E2E2E2E2000000E2E2E2E2A4
:102A40000000E2E2E2E2E200E2E2E2E2E200E2E2EE
:102A5000E2E2E2E2E2E2E2E2E2E2E2E2E2E2E2E256
:102A6000E2E2E2E2E2E2E2E2E2E20000E2E2E2E20A
:102A70000000E2E2E2E20000E2E2E2000000E2E264
:102A8000E2000000E2E2E2000000E2E2E2E2000036
:102A9000E2E2E2E200000000000000E200000000CC
:102AA000E2E2000000E2E2E2000000E2E2E2000016
:102AB00000E2E2E2000000E2E2E2000000E2E2E224
:102AC000000000E2E2E2E20000000000E2E20000BA
:102AD0000000E2E2E2000000E2E2E2000000E2E2E6
:102AE000E2000000E2E2E2000000E2E2E2000000B8
:102AF000E2E2E2000000E2E200000000E2E20000A8
:102B00000000E2E200000000E20000000000E2003D
:102B100000000000E20000000000E2E2000000000F
:102B2000E2E200000000000000E2E2E200E2E2E295
:102B3000E2E200E2E2E2E2E200E2E2E2E2E2E2E239
:102B4000E2E2E2E2E2E2E2E2E2E2E2E2E2E2E2E265
:102B5000E2E2E2E2E2E20000000000E20000000047
:102B600000E2E200000000E2E200000000E2E20019
:102B7000000000E2E200000000E2E200000000E2EB
:102B8000E200000000E2E200000000E2E2000000DB
:102B900000E2E200000000E2E200000000E2E200E9
:102BA000000000E2E200000000E2E200000000E2BB
:102BB000E200000000E2E2E2E2000000E2E2E20005
:102BC0000000E2E2E2000000E2E2E2000000E2E2F5
:102BD000E2000000E2E2E2000000E2E2E2000000C7
:102BE000E2E2E200000000E2E2E2E2E200E2E2E22F
:102BF000E2E200E2E2E2E2E200E2E2E2E2E200E25B
:102C0000E2E2E2E200E2E2E2E2E200E2E2E2E2E268
:102C100000E2E2E2E2E2000000E2E2E2000000E2C2
:102C2000E2E2000000E2E2E2000000E2E2E2000094
:102C300000E2E2E2000000E2E2E2000000E2E2E2A2
:102C4000000000E2E2E2E2E2E2E2E200E2E2E2E2EC
:102C5000E200E2E2E2E2E200E2E2E2E2E200E2E2FA
:102C6000E2E2E200E2E2E2E2E200E2E2E2E2E200EA
:102C7000E2E2E2E2E2000000E2E2E2E200E2E2E2BC
:102C8000E2E2E2E2E2E2E2E2E2E2E2E2E2E2E2E224
:102C9000E2E2E2E2E2E2E2E2E2E200E2E2E2E2E2F6
:102CA0000000E2E2E2E2E2E2E2E2E2E2E2E2E2E2C8
:102CB000E2E2E2E2E2E2E2E2E2E2E2E2E2E2E2E2F4
:102CC000E2E2E2E2E2E2E2E2E2E2E2E2E2E2E2E2E4
:102CD000E2E2E2E2E200E200000000E2E2000000E4
:102CE00000E2E200000000E2E200000000E200007A
:102CF000000000E20000000000E200000000000010
:102D0000000000000000E2E2E2E2E2E2E2E2E2E2EF
:102D1000E2E2E2E2E2E2E2E2E2E2E2E2E2E2E2E293
:102D2000E2E2E2E2E2E2E2E2E2E2E2E2E2E2E2E283
:102D300000E2E2E2E2E2E2E2E2E2E2E2E2E2E2E255
:102D4000E2E2E2E2E2E2E2E2E2E2E2E2E2E2E2E263
:102D5000E2E2E200E2E2E2E2E200E2E2E2E20000DB
:102D6000E2E2E200000000000000E2E200000000F9
:102D7000E2E200000000E2E200000000E2E2000007
:102D80000000E2E200000000E2E200000000E2E2F7
:102D90000000000000E2E2E200000000E2E20000C9
:102DA0000000E2E200000000E2E200000000E2E2D7
:102DB00000000000E20000000000E200000000004F
:102DC000E20000000000E2E2E2E20000E2E2E2E211
:102DD0000000E2E2E2E20000E2E2E2E20000E2E21F
:102DE000E2E2000000E2E2E2000000E2E2E20000D3
:102DF00000E2E2000000000000E2E2E2000000E287
:102E0000E2E2000000E2E2E2000000E2E2E20000B2
:102E100000E2E2E2000000E2E2E200000000E2E2A2
:102E20000000000000E2E2E2E2000000E2E2E20074
:102E30000000E2E2E2000000E2E2E2000000E2E282
:102E4000E2000000E2E2E2000000E2E20000000036
:102E5000E200000000000000E2E2E2E20000E2E244
:102E6000E2E20000E2E2E2E20000E2E2E2E200008E
:102E7000E2E2E2E20000E2E2E2E2000000E2E2E29C
:102E800000000000E2E2E2E200000000E2E20000F6
:102E90000000E2E200000000E2E200000000E2E2E6
:102EA00000000000E2E200000000E200000000007C
:102EB000000000000000E2E2E2E2E200E2E2E2E220
:102EC000E200E2E2E2E2E200E2E2E2E2E200E2E288
:102ED000E2E2E20000E2E2E2000000E2E2E2000000
:102EE00000E2E2E20000000000E2E2E2000000E2B4
:102EF000E2E2000000E2E2E2000000E2E2E20000C2
:102F000000E2E2E2000000E2E2E2000000E2E2E2CF
:102F100000000000E2E2E200000000E2E200000047
:102F200000E2E200000000E2E200000000E2E20055
:102F3000000000E2E20000000000E20000000000EB
:102F4000000000000000E2E2E2E20000E2E2E2E271
:102F50000000E2E2E2E20000E2E2E2E20000E2E29D
:102F6000E2E20000E2E2E2000000E2E2E200000051
:102F7000E2E2000000000000E2E2E2E20000E2E241
:102F8000E2E20000E2E2E2E20000E2E2E2E200006D
:102F9000E2E2E2E20000E2E2E2000000E2E2E2005D
:102FA000000000E2E200E2E2E2E2E2E2E2E2E2E289
:102FB000E2E2E2E2E2E2E2E2E2E2E2E2E2E2E2E2F1
:102FC000E2E2E2E2E2E2E2E2E2E2E2E2E2E2E2E2E1
:102FD000E2E2E2E2E2E2C2C2C2C2C2C2B2B2B2B251
:102FE000B2B2E2E2E2E2E2E2E2E2E2E2E2E2E2E221
:102FF000E2E2E2E2E2E2E2E2E2E2E2E2E2E2E2E2B1
:10300000E2E2E2E2E2E2E2E2E2E2E2E2E2E2E2E2A0
:10301000E2E2E2E2E2E2E2E2E2E2E2E2E2E2E2E290
:10302000E2E2E2E2E2E2E2E2E2E2B2B2B2B2B2B2A0
:10303000C2C2C2C2C2C2C2B2E2E2E2E2C2B2E2E2D0
:10304000E2E2C2B2E2E2E2E2C2B2E2E2E2E2C2B250
:10305000E2E2E2E2C2B2E2E2E2E2C2B2E2E2E2E2F0
:10306000C2B2E2E2E2E2E2E2E2E2B2C2E2E2E2E2E0
:10307000B2C2E2E2E2E2B2C2E2E2E2E2B2C2E2E220
:10308000E2E2B2C2E2E2E2E2B2C2E2E2E2E2B2C210
:10309000E2E2E2E2B2C2E2E2E2E2E2E2E2E2E2E260
:1030A000E2E2E2E2E2E2E2E2E2E2E2E2E2E2E2E200
:1030B000E2E2E2E2E2E2E2E2E2E2E2E2E2E2E2E2F0
:1030C000E2E2E2E2E2E2E2E2E2E2E2E2E2E2E2E2E0
:1030D000E2E2E2E2E2E2E2E2E2E2E2E2E2E2E2E2D0
:1030E000E2E2E2E2E2E2E2E2E2E2E2E2E2E2E2E2C0
:1030F000E2E2E2E2E2E2E2E2E2E2E2E2E2E2E2E2B0
:10310000E2E2E2E2E2E2E2E2E2E2E2E2E2E2E2E29F
:10311000E2E2E2E2E2E2E2E2E2E2E2E2E2E2E2E28F
:10312000E2E2E2E2E2E2E2E2E2E2E2E2E2E2E2E27F
:10313000E2E2E2E2E2E2E2E2E2E2E2E2E2E2E2E26F
:10314000E2E2E2E2E2E2E2E2E2E2E2E2E2E2E2E25F
:10315000E2E2E2E2E2E252525252525252525B5BDD
:103160005252525B52525B52525BAD5B5B52525BAE
:10317000AD5B5B52525B52525B5252525B5B52529E
:103180005252525252520000000707070000000737
:1031900007070000000707070000000707070707E9
:1031A00007000000070707000000070707000000EE
:1031B0000707070000000000000707070000C0C065
:1031C00007070000C0C0070700C0C0C0C00707C095
:1031D000C0C0C0000707C0C000000707C0C0000093
:1031E00007070700000002040202040204020202B0
:1031F00002040202020202020402020202040402A7
:103200000202020402020202020204020202020498
:103210000204020204020204020204020402020284
:1032200002040202C0C0020204C0C0C0C00404C044
:10323000C0C0C0040202C0C00202040202020204B2
:10324000020402020402FEFE1414FEFEFE14141414
:1032500014FEFE14141414FEFEFE1414FEFE0707E2
:1032600007070707070707070707140000000014F0
:10327000FE00FEFE00FE52F65252F65BF652A4A489
:1032800052F6F65B52525BF6525B525B5B52525BFC
:10329000AD525B52F65B52525BF6F652A4A452F664
:1032A0005BF65252F6520000002020200000002061
:1032B00020200000002020200000002020202020CE
:1032C000200000002020200000002020200000001E
:1032D0002020200000000000002020200000C0C0AE
:1032E00020200000C0C0202000C0C0C0C02020C0DE
:1032F000C0C0C0002020C0C000002020C0C000000E
:1033000020202000000038C0C0C0C0A0C0E080C0A5
:1033100080C0C0E0E49080C0C0E1E45080C0C0E064
:10332000E45080C0C0E1E4E480C0C0E0E1E0E1C07E
:10333000F8C0C0C0C03838C0C0C0C0A0C0E080C0A5
:1033400080C0C0E0070780C0C007070707C0C007EC
:10335000070707C0C0E1070780C0C0E0E1E0E1C0A7
:10336000F8C0C0C0C038FEFE3737FEFEFE37373724
:1033700037FEFE37373737FEFEFE3737FEFEA4A492
:10338000A4A4A4A4A4A4A4A4A4A437000000003767
:10339000FE00FEFE00FE3120504C415945520032E5
:1033A00020504C41594552004F5054494F4E5320E4
:1033B00000454449544F5220200032303039204CCF
:1033C0004545205745424552004C4556454C004224
:1033D0004554410050415553450054494C452D201A
:1033E0002D41542830302C30302900504C41595454
:1033F0004553542020200053415645284156522918
:1034000020200053415645285344292020200042C3
:1034100041434B20202020202020004558495420A3
:10342000454449544F520048454C5020202020200C
:103430002020005354415254202D204F50454E53CC
:10344000204D454E55202000414E442053454C45CB
:10345000435453204954454D532E20200020202012
:10346000202020202020202020202020202020205C
:10347000200042202D20504C414345532053454CC1
:103480004543544544200054494C45204154205460
:10349000484520435552534F52202000504F534926
:1034A00054494F4E2E484F4C442F44524147202000
:1034B00000544F20434F564552204C41524745201F
:1034C000415245415300582F59202D204348414E29
:1034D0004745532054484520202000504C41434547
:1034E0004D454E542054494C452E2020202020008C
:1034F000544F205445535420594F5552204C455653
:10350000454C20200043484F4F534520504C4159D3
:10351000544553542046524F4D005448452045448D
:1035200049544F52204D454E552E20544F200045B2
:1035300058495420544845204C4556454C20414656
:103540005445520054455354494E472C2048495441
:103550002053454C4543542000544F205245545568
:10356000524E20544F20454449544F522E00464558
:10357000454C204652454520544F20434F4E544120
:103580004354004D45204F4E2054484520464F524D
:10359000554D532E202020002D443354484144449F
:1035A00045522020202020202020202000202020E4
:1035B000202D484F5720544F20504C41592D20204A
:1035C0002000594F55522053494E474C4520474FF4
:1035D000414C2020202000495320544F2050555367
:1035E0004820424C4F434B5320202000414E442062
:1035F000434F56455220414C4C20544845202020F2
:1036000000544152474554532E20594F55204341B1
:103610004E275420200050554C4C204120424C4F06
:10362000434B2C20534F202020200054414B452059
:1036300043415554494F4E204E4F5420544F200083
:103640005055534820494E544F204120434F524E2D
:1036500045522E2000494620415420414E592054C5
:10366000494D4520594F552020004E454544205492
:103670004F2052455354415254204849542000533E
:10368000454C4543542E202020202020202020205F
:1036900020202000582F592057494C4C20524F547D
:1036A0004154452054484520004D41502E202020B3
:1036B000202020202020202020202020200020202A
:1036C00020202020202020202020202020202020FA
:1036D0002020002020204245544120564552534985
:1036E0004F4E2020202020005448414E4B5320466E
:1036F0004F5220504C4159494E472E20004F5054B4
:10370000494F4E5320200054494C4553202020203F
:1037100000534F4B4F42414E2020004C4556454CE4
:10372000202020200048454C50202020202000450B
:103730005849542020202020004D55534943202033
:10374000202000474F544F204C4556454C20202008
:1037500000534F4B4F42414E202020202020005448
:10376000494C45532020202020202020004D555337
:10377000494320202020202020200052455354413E
:103780005254204C4556454C004241434B2020208A
:10379000202020202020004558495420544F2054F8
:1037A00049544C45004F4646004C4F534520554E1A
:1037B00053415645443F00594553004E4F200000A9
:1037C00000000000000000000000000000000000F9
:1037D00000000000000000000000000000000000E9
:1037E00000000000000000000000000000000000D9
:1037F00000E2E2E2E200E2E2E2E2E200E2E2E2E24F
:10380000E200E2E2E2E2E2E2E2E2E2E2E2E2E2E27A
:10381000E2E2E2E2E2E2E2E2E2E2E2E2E2E2E2E288
:10382000E2E2E2E200E2E2E2E2E2E2E2E2E2E2E25A
:10383000E2E2E2E2E2E2E2E2E2E2E2E2E2E2E2E268
:10384000E2E2E2E2E2E2E2E2E2E2E2E2E2E200001C
:103850000000000000000000000000E20000000086
:1038600000E20000000000E20000000000E20000B2
:103870000000000000000000000000000000000048
:103880000000000000000000000000000000000038
:103890000000000000000000000000000000000028
:1038A0000000000000000000000000000000000018
:1038B00000000000E200000000E2E200000000E280
:1038C000E200000000E2E200000000E2E20000008E
:1038D00000E2E200000000E2E200000000E2E2E2BA
:1038E0000000000000E20000000000E20000000014
:1038F00000E2E200000000E2E200000000E2E2007C
:10390000000000E2E200000000E2E200000000002F
:10391000E2E200000000E2E2E2000000E2E2E20097
:1039200000E2E2E2E20000E2E2E2E20000E2E2E2E1
:10393000E20000E2E2E2E20000E2E2E2E200000095
:10394000000000E2E2000000E2E2E20000E2E2E267
:10395000E20000E2E2E2E20000E2E2E2E20000E293
:10396000E2E2E20000E2E2E2E20000E2E2E2E2E2BF
:10397000E2E2E2E2E2E2E2E2E2E2E2E2E2E2E2E227
:10398000E2E2E2E2E2E2E2E2E2E2E2E2E2E2E2E217
:10399000E2E2E2E2E2E2E2E2E2E2E2E2E2E2E200E9
:1039A0000000000000E20000000000E2E200000071
:1039B00000E2E200000000E2E200000000E2E200BB
:1039C000000000E2E200000000E2E200000000006F
:1039D00000000000000000000000000000000000E7
:1039E000000000000000000000000000E2000000F5
:1039F0000000E20000000000E20000000000E20021
:103A0000E2E2E2E2E2E2E2E2E2E2E2E2E2E2E2E296
:103A1000E2E2E2E2E2E2E2E2E2E2E2E2E2E2E2E286
:103A2000E2E2E2E2E2E2E2E2E2E2E2E2E2E2E2E276
:103A3000E2E2E20000E2E2E2E2E200E2E2E2E2E20C
:103A400000E2E2E2E2E200E2E2E2E2E2E2E2E2E21A
:103A5000E2E2E2E2E2E2E2E2E2E2E2E2E2E2E2E246
:103A6000E2E2E20000E2E2E2E20000E2E2E2E200A0
:103A700000E2E2E2E20000E2E2E2E20000E2E2E290
:103A8000E20000E2E2E2E20000E2E2E2E200000044
:103A9000000000E2E200000000E2E200000000E2BC
:103AA000E200000000E2E200000000E2E2000000AC
:103AB00000E2E200000000E2E200000000E2E2E2D8
:103AC000E200000000E2E200000000E2E20000008C
:103AD00000E2E200000000E2E200000000E2E2009A
:103AE000000000E2E200000000E2E200000000004E
:103AF00000E2E2E2E20000E2E2E2E20000E2E2E210
:103B0000E20000E2E2E2E20000E2E2E2E20000E2E1
:103B1000E2E2E20000E2E2E2E20000E2E2E2E200EF
:103B200000000000E20000000000E20000000000D1
:103B3000E20000000000E20000000000E2000000DF
:103B40000000E20000000000E20000000000E2E2ED
:103B5000E2E2E2E2E2E2E2E2E2E2E2E2E2E2E2E245
:103B6000E2E2E2E2E2E2E200E2E2E2E2E200E2E2F9
:103B7000E2E2E200E2E2E2E2E20000E2E2E2E2E2CB
:103B8000E2E2E2E200E2E2E2E2E2E2E2E2E2E2E2F7
:103B9000E2E2E2E2E2E2E2E2E2E2E2E2E2E2E2E205
:103BA000E2E2E2E2E2E2E2E2E2E2E2E2E2E2E200D7
:103BB0000000000000000000000000000000000005
:103BC000E20000000000E2E200000000E2E200008B
:103BD0000000E2E200000000E2E200000000E2E299
:103BE000E2E2000000E2E2E2E20000E2E2E2E2E21F
:103BF00000E2E2E2E2E200E2E2E2E2E2E2E2E2E269
:103C0000E2E2E2E2E2E2E2E2E2E2E2E2E2E2E2E294
:103C1000E2E2E20000E2E2E2E20000E2E2E2E200EE
:103C200000E2E2E2000000E2E2E2000000E2E2E2A2
:103C3000000000E2E2E2E20000E2E2E2E200000074
:103C400000000000E200000000E2E2000000E2E20A
:103C5000E2000000E2E2E2000000E2E2E200000036
:103C6000E2E2E2000000E2E2E2000000E2E2E2E280
:103C70000000000000E2E200000000E2E2E20000DA
:103C800000E2E2E2000000E2E2E2000000E2E2E242
:103C9000000000E2E2E2000000E2E2E2000000E2F6
:103CA000E200000000E2E200000000E2E2000000AA
:103CB00000E20000000000E20000000000E200005E
:103CC000000000E2E200000000E2E200000000006C
:103CD0000000E2E2E200E2E2E2E2E200E2E2E2E24C
:103CE000E200E2E2E2E2E2E2E2E2E2E2E2E2E2E296
:103CF000E2E2E2E2E2E2E2E2E2E2E2E2E2E2E20086
:103D000000000000E20000000000E2E2000000000D
:103D1000E2E200000000E2E200000000E2E2000057
:103D20000000E2E200000000E2E200000000E2E247
:103D300000000000E2E200000000E2E200000000FB
:103D4000E2E200000000E2E200000000E2E2000027
:103D50000000E2E200000000E2E200000000E2E217
:103D6000E2E2000000E2E2E2000000E2E2E2000043
:103D700000E2E2E2000000E2E2E2000000E2E2E251
:103D8000000000E2E2E2000000E2E2E200000000E7
:103D9000E2E2E2E2E200E2E2E2E2E200E2E2E2E2C7
:103DA000E200E2E2E2E2E200E2E2E2E2E200E2E299
:103DB000E2E2E200E2E2E2E2E200E2E2E2E2E20089
:103DC0000000E2E2E2000000E2E2E2000000E2E2E3
:103DD000E2000000E2E2E2000000E2E2E2000000B5
:103DE000E2E2E2000000E2E2E2000000E2E2E2E2FF
:103DF000E2E2E2E200E2E2E2E2E200E2E2E2E2E267
:103E000000E2E2E2E2E200E2E2E2E2E200E2E2E238
:103E1000E2E200E2E2E2E2E200E2E2E2E2E200000A
:103E200000E2E2E2E200E2E2E2E2E2E2E2E2E2E236
:103E3000E2E2E2E2E2E2E2E2E2E2E2E2E2E2E2E262
:103E4000E2E2E200E2E2E2E2E20000E2E2E2E2E2F8
:103E5000E2E2E2E2E2E2E2E2E2E2E2E2E2E2E2E242
:103E6000E2E2E2E2E2E2E2E2E2E2E2E2E2E2E2E232
:103E7000E2E2E2E2E2E2E2E2E2E2E2E2E2E200E204
:103E800000000000E2E200000000E2E200000000AA
:103E9000E2E200000000E20000000000E20000009A
:103EA0000000E2000000000000000000000000E24E
:103EB000E2E2E2E2E2E2E2E2E2E2E2E2E2E2E2E2E2
:103EC000E2E2E2E2E2E2E2E2E2E2E2E2E2E2E2E2D2
:103ED000E2E2E2E2E2E2E2E2E200E2E2E2E2E2E2A4
:103EE000E2E2E2E2E2E2E2E2E2E2E2E2E2E2E2E2B2
:103EF000E2E2E2E2E2E2E2E2E2E2E2E200E2E2E284
:103F0000E2E200E2E2E2E20000E2E2E200000000BF
:103F1000000000E2E200000000E2E200000000E237
:103F2000E200000000E2E200000000E2E200000027
:103F300000E2E200000000E2E20000000000E2E235
:103F4000E200000000E2E200000000E2E200000007
:103F500000E2E200000000E2E200000000E20000F7
:103F6000000000E20000000000E20000000000E2AB
:103F7000E2E2E20000E2E2E2E20000E2E2E2E2008B
:103F800000E2E2E2E20000E2E2E2E2000000E2E25D
:103F9000E2000000E2E2E2000000E2E200000000D5
:103FA0000000E2E2E2000000E2E2E2000000E2E201
:103FB000E2000000E2E2E2000000E2E2E2000000D3
:103FC000E2E2E200000000E2E20000000000E2E2C3
:103FD000E2E2000000E2E2E2000000E2E2E20000D1
:103FE00000E2E2E2000000E2E2E2000000E2E2E2DF
:103FF000000000E2E200000000E20000000000001B
:1040000000E2E2E2E20000E2E2E2E20000E2E2E2FA
:10401000E20000E2E2E2E20000E2E2E2E20000E2CC
:10402000E2E2E2000000E2E2E200000000E2E2E29E
:10403000E200000000E2E200000000E2E200000016
:1040400000E2E200000000E2E200000000E2E20024
:10405000000000E20000000000000000000000E29C
:10406000E2E2E2E200E2E2E2E2E200E2E2E2E2E2F4
:1040700000E2E2E2E2E200E2E2E2E2E20000E2E2A8
:10408000E2000000E2E2E2000000E2E2E200000002
:104090000000E2E2E2000000E2E2E2000000E2E210
:1040A000E2000000E2E2E2000000E2E2E2000000E2
:1040B000E2E2E2000000E2E2E200000000E2E2E20E
:1040C00000000000E2E200000000E2E20000000068
:1040D000E2E200000000E2E200000000E2E2000094
:1040E000000000E20000000000000000000000E20C
:1040F000E2E2E20000E2E2E2E20000E2E2E2E2000A
:1041000000E2E2E2E20000E2E2E2E20000E2E2E2F9
:10411000000000E2E2E2000000E2E2000000000035
:1041200000E2E2E2E20000E2E2E2E20000E2E2E2D9
:10413000E20000E2E2E2E20000E2E2E2E20000E2AB
:10414000E2E2000000E2E2E200000000E2E200C77A
:10415000C7C7C7C7C7C7C7C7C7C7C7C7C7C7C7C7EF
:10416000C7C7C7C7C7C7C7C7C7C7C7C7C7C7C7C7DF
:10417000C7C7C7C7C7C7C7C7C7C7C7C7C7C7C71383
:10418000068788898A8A8B8C8D8A8A8A8E8F908A04
:104190008A919293948A8A8A8A9596948A8A8A972F
:1041A00095968A8A989497999A9B929C958F9D9EB2
:1041B0008F9F978FA0A19AA294978A97A3A4A59561
:1041C0009694A6A3A4979596A7A6A394978A97A337
:1041D000A4A5959694A6A3A49795968F8FA394973C
:1041E000A8A9AAABACADAEAFB08FB1B28FB3B4B526
:1041F000B6B7B80808464748494A4B4C4D56575839
:10420000595A5B5C5D666768696A6B6C6D76777836
:10421000797A7B7C7D4E4F5051525354555E5F608E
:1042200061626364656E6F7071727374757E7F8096
:10423000818283848508084E4F5051464748495E25
:104240005F6061565758596E6F7071666768697E16
:104250007F808176777879525354554A4B4C4D6222
:104260006364655A5B5C5D727374756A6B6C6D82B6
:104270008384857A7B7C7D0808525354554E4F5079
:1042800051626364655E5F6061727374756E6F70B6
:1042900071828384857E7F80814A4B4C4D4647489E
:1042A000495A5B5C5D565758596A6B6C6D66676816
:1042B000697A7B7C7D7677787908084A4B4C4D5239
:1042C0005354555A5B5C5D626364656A6B6C6D72D6
:1042D0007374757A7B7C7D82838485464748494E1A
:1042E0004F5051565758595E5F6061666768696EF6
:1042F0006F7071767778797E7F8081040401020384
:104300000405060708090A0A0B0C0D0E0F00020629
:104310000000FB00FF0000F405030605040605038A
:104320000605040605050000FF00FF000209000065
:10433000F10400F900FF00010A0000E2020105019A
:10434000010301010102050000FF0000E702030C68
:1043500004050000FF0000F100085A0204030204F3
:104360000402040502040602050000FF000101002A
:1043700007900000E208050000FF0002080107C8DE
:104380000106000100E700FF0001000007A0000097
:10439000EC0100FE00010100FF0001030000E20348
:1043A000010604010903050000FF0002010107C81E
:1043B0000106000100EC00FF0002040000F104000F
:1043C000F900FF0002010000F100FF0000ED000114
:1043D0000602010100FF0000EC00010201070002DB
:1043E00007FF00010300FF0002080007640100143A
:1043F0000500F700FF0002090000F100FF000204C1
:104400000000F800085003084E03085402084C024C
:10441000085802084A01085C0000FC030860030811
:104420005A03086003085A03086003085A0105008C
:1044300000FF0002040000FB00083E01030201032C
:104440000201030201030201030201040A01030243
:10445000010302010302010302010302010402013C
:10446000030201030201030201030201030201042A
:104470000A01030201030201030201030201030214
:104480000104050103020103020103020103020109
:1044900003020104050103020103020103020103F7
:1044A00002010302010405010302010302010302E8
:1044B00001030201030201050000FF0002030008DE
:1044C0005602040A0204080204060204040204025A
:1044D000000842020305020402020305020305026A
:1044E00004020203050000F80403050404050403A4
:1044F000050404050403050404050403050105007F
:1045000000FF0002040000FB000834010302010365
:104510000401030601040A01030201030401030666
:1045200001040A0103020103040103060104050159
:10453000030201030401030602030202030402034F
:10454000060304050303020303040303060404052E
:1045500004030204030404030601050000FF00072E
:10456000000402040007FF000990000A3C0000FB61
:1045700001085003030503040503030503040503B1
:1045800003050304050303050304050303050304EE
:104590000503030503040503030503050000FF00ED
:1045A00007000402040007FF000990000A3C000015
:1045B000FB01085303030503040503030503040576
:1045C00003030503040503030503040503030503AF
:1045D000040503030503040503030503050000FFA9
:1045E0000007000402040007FF000990000A3C00D5
:1045F00000FB010856030305030405030305030438
:10460000050303050304050303050304050303056C
:104610000304050303050304050303050305000064
:10462000FF0007000402040007FF000990000A3C95
:104630000000FB01085903030503040503030503F8
:10464000040503030503040503030503040503032D
:10465000050304050303050304050303050305001F
:1046600000FF0002020106000100E000FF0002015D
:104670000106000100E000FF000208010600010041
:10468000E000FF0002050106000100E000FF00025B
:10469000090106000100E000FF0000000D430000DA
:1046A0000000000000154300000000000000294346
:1046B000000000000000002B43000000000100008B
:1046C0003643000000000000004A430000000000E4
:1046D00000005543000000000100006C4300000092
:1046E000000000007A430000000001000088430041
:1046F000000000010000994300000000000000AA33
:104700004300000000000000B8430000000000006B
:1047100000C34300000000010000CB430000000084
:10472000010000D64300000000000000E743000045
:104730000000000000F54300000000000000FD4301
:1047400000000000000000324400000000000000F3
:10475000BB44000000000000000245000000000013
:1047600000005E45000000000000009F45000000C2
:1047700000000000E04500000000000000214600AD
:104780000000000000006246000000000000006D14
:104790004600000000000000784600000000000015
:1047A000008346000000000000008E46000000006C
:1047B00000FF06015300C00000904C6B00C20000D7
:1047C00092286B00C1000091476B1792346B1890D0
:1047D000476B0092286B0091446B1890486B0092D5
:1047E000346B0091456B18904A6B0092286B0091D6
:1047F000476B18904C6B0092346B0091446B0C909B
:104800004A6B0C486B0092286B0091456B189047DF
:104810006B0092346B0091446B1890456B00922DA5
:104820006B0091406B1892396B1890456B00922D7C
:104830006B0091406B1890486B0092396B0091456A
:104840006B18904C6B00922D6B0091486B1892394D
:104850006B18904A6B00922D6B0091476B18904833
:104860006B0092396B0091456B1890476B00922C4E
:104870006B0091446B1892386B1890476B00922C28
:104880006B0091446B1890486B0092386B00914517
:104890006B18904A6B0092286B0091476B1892340A
:1048A0006B18904C6B0092286B0091476B189234F8
:1048B0006B1890486B00922D6B0091456B189239E4
:1048C0006B1890456B00922D6B0091406B189239DC
:1048D0006B1890456B00922D6B0091406B189239CC
:1048E0006B182D6B00912F6B1892306B0091396B08
:1048F0001892266B0091326B18904A6B0092326BC3
:104900000091456B1892266B18904D6B0092326B9C
:1049100000914A6B1890516B0092266B00914D6B81
:104920001892326B18904F6B0092266B00914C6B73
:1049300018904D6B0092326B00914A6B18904C6B43
:1049400000922D6B0091486B1892396B182D6B18E3
:1049500090486B0092396B0091456B18904C6B003E
:10496000922D6B0091456B1892396B18904A6B0031
:10497000922D6B0091476B1890486B0092396B0039
:1049800091456B1890476B00922C6B0091446B180B
:1049900092386B1890476B00922C6B0091446B1807
:1049A00090486B0092386B0091456B18904A6B00F1
:1049B00092286B0091476B1892346B18904C6B00E7
:1049C00092286B0091476B1892346B1890486B00DB
:1049D000922D6B0091456B1892396B1890456B00C6
:1049E000922D6B0091406B1892396B1890456B00BB
:1049F000922D6B0091406B1892396B182D6B183902
:104A00006B18904C6B0092286B0091476B18923496
:104A10006B1790476B0092286B0091446B1890487D
:104A20006B0092346B0091456B18904A6B00922892
:104A30006B0091476B18904C6B0092346B00914463
:104A40006B0C904A6B0C486B0092286B0091456B85
:104A50001890476B0092346B0091446B1890456B33
:104A600000922D6B0091406B1892396B1890456B3A
:104A700000922D6B0091406B1890486B0092396B3F
:104A80000091456B18904C6B00922D6B0091486B18
:104A90001892396B18904A6B00922D6B0091476BFE
:104AA0001890486B0092396B0091456B1890476BDA
:104AB00000922C6B0091446B1892386B1890476BE6
:104AC00000922C6B0091446B1890486B0092386BED
:104AD0000091456B18904A6B0092286B0091476BD0
:104AE0001892346B18904C6B0092286B0091476BB6
:104AF0001892346B1890486B00922D6B0091456BA7
:104B00001892396B1890456B00922D6B0091406B99
:104B10001892396B1890456B00922D6B0091406B89
:104B20001892396B182D6B00912F6B1892306B0017
:104B300091396B1892266B0091326B18904A6B007A
:104B400092326B0091456B1892266B18904D6B005A
:104B500092326B00914A6B1890516B0092266B0059
:104B6000914D6B1892326B18904F6B0092266B0030
:104B7000914C6B18904D6B0092326B00914A6B1800
:104B8000904C6B00922D6B0091486B1892396B180A
:104B90002D6B1890486B0092396B0091456B189003
:104BA0004C6B00922D6B0091456B1892396B1890ED
:104BB0004A6B00922D6B0091476B1890486B0092E6
:104BC000396B0091456B1890476B00922C6B0091EC
:104BD000446B1892386B1890476B00922C6B0091C5
:104BE000446B1890486B0092386B0091456B18909D
:104BF0004A6B0092286B0091476B1892346B1890A7
:104C00004C6B0092286B0091476B1892346B189094
:104C1000486B00922D6B0091456B1892396B189080
:104C2000456B00922D6B0091406B1892396B189078
:104C3000456B00922D6B0091406B1892396B182DCB
:104C40006B18396B1890406B00922D6B00913C6B88
:104C50001892346B182D6B17346B18903C6B0092C4
:104C60002D6B0091396B1892346B182D6B18346BC7
:104C700018903E6B00922C6B0091386B1892346B3D
:104C8000182C6B18346B18903B6B00922C6B0091B6
:104C9000386B1892346B182C6B18346B18903C6B73
:104CA00000922D6B0091396B1892346B182D6B1894
:104CB000346B182D6B0091396B1892346B182D6B77
:104CC00018346B182C6B0091386B1892346B182CBD
:104CD0006B18346B182C6B18346B182C6B18346BE6
:104CE0001890406B00922D6B00913C6B1892346BC6
:104CF000182D6B18346B18903C6B00922D6B009143
:104D0000396B1892346B182D6B18346B18903E6BFE
:104D100000922C6B0091386B1892346B182C6B1826
:104D2000346B18903B6B00922C6B0091386B18928F
:104D3000346B182C6B18346B18903C6B00922D6BF5
:104D40000091396B1892346B1890406B00922D6B68
:104D500000913C6B1892346B1890456B00922D6B50
:104D60000091406B1892346B1890456B00922D6B3C
:104D700018346B1890446B00922C6B0091406B18A8
:104D800092346B182C6B18346B182C6B18346B180E
:104D90002C6B18346B18FF06014500FF2F00000034
:104DA0000000000000000000000000000000000003
:104DB00000000000000000000000000000000000F3
:104DC00000000000000000000000000000000000E3
:104DD00000000000000000000000000000000000D3
:104DE00000000000000000000000000000000000C3
:104DF00000000000000000010101010100000000AE
:104E0000000000000000000000000000010202029B
:104E10000100000000000000000000000000000091
:104E20000001040202010000000000000000000078
:104E30000000000001010102020401010000000065
:104E40000000000000000000000102020402040251
:104E5000010000000000000000000000010101024C
:104E60000102010102010000000101010101010034
:104E7000000102020201020101020101010101021D
:104E80000203030100000102040202040202020202
:104E900002020202020203030100000101010101FA
:104EA00002010101020106010102020303010000E7
:104EB00000000000010202020202010101010101E1
:104EC00001010100000000000001010101010101D8
:104ED00000000000000000000000000000000000D2
:104EE00000000000000000000000000000000000C2
:104EF00000000000000000000000000000000000B2
:104F000000000000000000000000000000000000A1
:104F10000000000000000000000000000000000091
:104F20000000000000000000000000000000000081
:104F30000000000000000000000000000000000071
:104F40000000000000000000000000000000000061
:104F50000000000000000000000000000000000051
:104F60000000000000000000000000000000000041
:104F70000000000000000000000000000000000031
:104F80000000000000000000000000000000000021
:104F90000000000000000000000000000000000011
:104FA0000000000000000000000000000000000001
:104FB00000000000000000000000000000000000F1
:104FC00000000001010101010101010101010100D5
:104FD00000000000000000000103030202010202C1
:104FE00002020201010100000000000000010303B1
:104FF0000202010204020204020201000000000099
:105000000000010303020201040101010102020187
:105010000000000000000001030302020202020679
:105020000101020201000000000000000103030270
:10503000020102010202040201010000000000005E
:105040000001010101010102010104020402010049
:10505000000000000000000001020402020402043B
:105060000204020100000000000000000001020232
:105070000202010202020202010000000000000020
:105080000000010101010101010101010101000014
:105090000000000000000000000000000000000010
:1050A0000000000000000000000000000000000000
:1050B00000000000000000000000000000000000F0
:1050C00000000000000000000000000000000000E0
:1050D00000000000000000000000000000000000D0
:1050E00000000000000000000000000000000000C0
:1050F00000000000000000000000000000000000B0
:10510000000000000000000000000000000000009F
:10511000000000000000000000000000000000008F
:10512000000000000000000000000000000000007F
:10513000000000000000000000000000000000006F
:10514000000000000000000000000000000000005F
:10515000000000000000000000000000000000004F
:10516000000000000000000000000000000000003F
:10517000000000000000000000000000000000002F
:105180000000000101010101010101000000000017
:1051900000000000000000000102020202020601FD
:1051A00000000000000000000000000000010204F8
:1051B00001040201010000000000000000000000E6
:1051C00000000102040202040100000000000000CF
:1051D00000000000000000010104020402010000C0
:1051E00000000000010101010101010101020402AE
:1051F0000102010101000000000103030303020298
:105200000101020402020402020100000000010187
:10521000030303020202020402020402020201006A
:105220000000000103030303020201010101010167
:105230000101010100000000010101010101010162
:10524000000000000000000000000000000000005E
:10525000000000000000000000000000000000004E
:10526000000000000000000000000000000000003E
:10527000000000000000000000000000000000002E
:10528000000000000000000000000000000000001E
:10529000000000000000000000000000000000000E
:1052A00000000000000000000000000000000000FE
:1052B00000000000000000000000000000000000EE
:1052C00000000000000000000000000000000000DE
:1052D00000000000000000000000000000000000CE
:1052E00000000000000000000000000000000000BE
:1052F00000000000000000000000000000000000AE
:10530000000000000000000000000000000000009D
:10531000000000000000000000000000000000008D
:10532000000000000000000000000000000000007D
:10533000000000000000000000000000000000006D
:10534000000000000000000000000000000101015A
:105350000101010100000000000000000000000049
:105360000000010202030202010000000000000030
:105370000000000001010101030103040401010117
:10538000010000000000000000010302020202030D
:1053900001020204060100000000000000000102FA
:1053A00004020201020202020402010000000000E5
:1053B00000000001010101020405010201030101D5
:1053C00000000000000000000000000102020202D4
:1053D00002010101000000000000000000000000C8
:1053E00001010101010101000000000000000000B6
:1053F00000000000000000000000000000000000AD
:10540000000000000000000000000000000000009C
:10541000000000000000000000000000000000008C
:10542000000000000000000000000000000000007C
:10543000000000000000000000000000000000006C
:10544000000000000000000000000000000000005C
:10545000000000000000000000000000000000004C
:10546000000000000000000000000000000000003C
:10547000000000000000000000000000000000002C
:10548000000000000000000000000000000000001C
:10549000000000000000010000000000000000000B
:1054A00000000000000000000000000100000000FB
:1054B00000000000000000000000000000000000EC
:1054C00001000000000000000101010101010101D3
:1054D00000000000000100000000000000010202C6
:1054E00002020202010000000000010000000000B2
:1054F00000010102010101010201000000000001A0
:10550000000000000000010302030103010201008A
:105510000000000001000000000000010202020281
:105520000202020100000000000100000000010171
:105530000101040404020202010000000000010055
:10554000000000010202030406040301010100003F
:105550000000000100000000010201010404040237
:105560000202010000000000010000000001020131
:10557000020202020202020100000000000100001B
:105580000000010201030203020301020100000006
:1055900000000100000000010202020201020101FC
:1055A00002010000000000010000000001010101F3
:1055B00001010202020201000000000001000000DF
:1055C00000000000000001010101010100000000D5
:1055D00000010000000000000000000000000000CA
:1055E00000000000000001000000000000000000BA
:1055F00000000000000000000000000100000000AA
:10560000000000000000000000000000000000009A
:105610000100000000000000000000000000000089
:105620000000000000010000000000000000000079
:105630000000000000000000000001000000000069
:10564000000000000000000000000000000000005A
:10565000000000000000000000000000000000004A
:10566000000000000000000000000000000000003A
:10567000000000000000000000000000000000002A
:10568000000000000000000000000000000000001A
:105690000000000000000001010100000000000007
:1056A00000000000000000000000000102020201F2
:1056B00000000000000000000000000000000001E9
:1056C00003030203030100000000000000000000CB
:1056D00000000101010402040204010101000000B4
:1056E00000000000000000010202020302030202A7
:1056F00002010000000000000000000001020101A2
:10570000020102010102010000000000000000008F
:105710000001020202040204020202010000000071
:105720000000000000000102010402030204010263
:10573000010000000000000000000001020203045C
:10574000010403020201000000000000000000004C
:10575000010101010202020101010100000000003B
:10576000000000000000000001010601010000002F
:105770000000000000000000000000000000010127
:105780000101000000000000000000000000000017
:105790000000000000000000000000000000000009
:1057A00000000000000000000000000000000000F9
:1057B00000000000000000000000000000000000E9
:1057C00000000000000000000000000000000000D9
:1057D00000000000000000000000000000000000C9
:1057E00000000000000000000000000000000000B9
:1057F0000000000000800320038020802020402043
:105800002003400D100D20802020400E10072003A3
:10581000802080202003408080202003400B104007
:10582000108020801010202040062003802020803F
:105830002003408080202003400B104010802080F7
:105840001040072003802020038020054080802016
:105850002003400B108010402040101020208006B4
:1058600020038020200380100340202004400310E8
:1058700003802020802003408080202003400B10E4
:10588000801040204010FF01401010034010108095
:1058900080208080108080202080042040408080F4
:1058A000041040101040402040032080062080203B
:1058B000400510038010104020802040408080046C
:1058C00010401010404020400320800620041003A8
:1058D000800410400320802040408006104040207B
:1058E0004003208005208020400610400310808067
:1058F0001080052080204040800510034003208058
:105900000520051040031040104040200380100384
:105910008010800520802040408005100340032037
:10592000800520402080108020201010400410406E
:10593000031040402080100480052040401010409B
:10594000101040100380108005208020404080050A
:105950001003400320800420402080108020400558
:1059600010401010034020208010104010058010BF
:1059700080052080204040800510034003208004E3
:1059800020402080801080202010104040041040D3
:1059900010401040402020801010401005801080E2
:1059A00005208020404080051040404003208004B6
:1059B00020402080801080204040031003400410CD
:1059C0004010058010800520802040408005100395
:1059D00040032080052040200380108020201010EC
:1059E000034010100440032080101040100380403A
:1059F00040031080802080042040200380108020FD
:105A0000FF02200340802020044008208020401016
:105A100040200410800510801010400A2080204093
:105A2000091004800210402080200340104008200C
:105A300080204008100480101080802040401040DA
:105A40002080200440104009200C108020208080FD
:105A500020808010044010400920802040071080E2
:105A6000102080801010404010400A200510801047
:105A700040101010808080202040401040072004FB
:105A8000108080104003108080202040401040068D
:105A9000204020801080042004104007100680045D
:105AA0002040400310801004401040082040208017
:105AB0001080032003104005100480200340104094
:105AC0000520402080108020201010400710068004
:105AD0000320054010400520402080108020FF005A
:105AE00011241FBECFEFD0E1DEBFCDBF14BE88E1D1
:105AF0000FB6F89480936000109260000FBE13E020
:105B0000A0E0B1E0EEE0F7EB02C005900D92AC35FD
:105B1000B107D9F71FE0A0E6B3E001C01D92A430A1
:105B2000B107E1F7F894E1E6F3E080E090E020E8E7
:105B300002C02193019632E08C309307D4F381E6C2
:105B400093E090936E0580936D0510926F05E2E7E8
:105B5000F5E080E090E003C0108201963A96843030
:105B60009105D4F381E0809392058093930580930F
:105B700091051092810015BCE0E0F1E080E090E03A
:105B80002EEF02C02193019680399105DCF39093AA
:105B9000780E8093770E80E00E948442E0E0FAE085
:105BA00080E090E050ED20EA35E041E00EC0108248
:105BB0001182009719F45093020A01C012823483B3
:105BC00023831782408701963F96181619067CF7A3
:105BD0009093780E8093770E91E09093270E8FEF3D
:105BE00087B984B980E88AB98CE081B983EF82B93A
:105BF0001092280E86E08093290E10928500109254
:105C0000840083E0809389008DE88093880089E098
:105C10008093810082E080936F0082E484BD17BC92
:105C200095BD83E88093B0001092B3009093B100CB
:105C300081E185B978940E94232E0E9428590C9402
:105C4000855B0C9400001F9387E59BE00E94672F03
:105C500084E990E09093060A8093050A0E945A42D4
:105C60008FE090E00E946C3B87E59BE00E94672FED
:105C700088E290E00E946C3B80E16CE044EE5AE0E8
:105C80000E940C3C84E090E00E946C3B0E945A42CF
:105C90008CE06CE044EE5AE00E940C3C84E090E022
:105CA0000E946C3B0E945A428AE06CE044EE5AE04B
:105CB0000E940C3C84E090E00E946C3B0E945A429F
:105CC00088E06CE044EE5AE00E940C3C86E090E0F4
:105CD0000E946C3B88E06CE048E15BE00E940C3C79
:105CE0008AE090E00E946C3B88E06CE044EE5AE071
:105CF0000E940C3C8EE190E00E946C3B18E00E94F8
:105D00005A42812F6CE044EE5AE00E940C3C86E03F
:105D100090E00E946C3B115090F710E00E945A42B4
:105D2000112329F480E06CE044EE5AE004C0812F96
:105D30006CE048E15BE00E940C3C812F84506CE0F9
:105D400040E750E00E940C3C86E090E00E946C3BF3
:105D50001E5F183019F710E00E945A42113138F4D2
:105D6000812F885F6CE044EE5AE00E940C3C812F4A
:105D70008C5F6CE040E750E00E940C3C86E090E0D5
:105D80000E946C3B1E5F143139F710E00E945A42AA
:105D900088E0612F44EE5AE00E940C3C1F5F82E0D5
:105DA00090E00E946C3B1C3089F788E06BE048E192
:105DB0005BE00E940C3C80E06FEF41E00E94F83213
:105DC00086E090E00E946C3B88E06BE044EE5AE095
:105DD0000E940C3C86E090E00E946C3B88E06BE007
:105DE00048E15BE00E940C3C86E090E00E946C3B46
:105DF00088E06BE044EE5AE00E940C3C84E190E0C5
:105E00000E946C3B80E590E00E946C3B0E945A42ED
:105E100084E190E00E946C3B1F91089590E025E1A1
:105E200030E0829FF001839FF00D929FF00D1124CE
:105E3000E558F14F6187089560939105089590E0CA
:105E400025E130E0829FF001839FF00D929FF00DDD
:105E50001124E558F14F12861182089590E025E152
:105E600030E0829FF001839FF00D929FF00D11248E
:105E7000E558F14F81E0828B089590E025E130E014
:105E8000829FF001839FF00D929FF00D1124E55841
:105E9000F14F6087089590E025E130E0829FF001A6
:105EA000839FF00D929FF00D1124E558F14F64830C
:105EB000089590E025E130E0829FF001839FF00D8E
:105EC000929FF00D1124E558F14F6583089590934A
:105ED000D20E8093D10E8FE68093D70E109260037E
:105EE000EBE7FEE021E09FEF88E1208317829683B5
:105EF00013861182858375963EE0EF3CF307A9F780
:105F0000089510927C0E1092910E1092A60E10928F
:105F1000BB0E01969093DB0E8093DA0E90937A0E6F
:105F20008093790E9093DE0E8093DD0E1092D90E41
:105F30001092D80E1092D00E1092CF0E1092D30E57
:105F400081E0809360031092D60E1092D50E0895D2
:105F50008091790E90917A0E0E94812F08958AEF98
:105F60008093840E8093990E8093AE0E8093C30E1F
:105F700010926003089581E0809360030895DC012E
:105F8000ED91FC911197AF014F5F5F4F11965C93BC
:105F90004E93E4912E2F30E0E7FF13C02F7730703F
:105FA0003695322F222737952795FA014F5F5F4F9D
:105FB000E4918E2F8F77280F311DE7FDF1CF4D93A0
:105FC0005C93C90108958093D70E089508950E94A7
:105FD0001F340895EF92FF920F931F93CF93DF9397
:105FE000182F062FF42EE22EC82FD0E085E190E086
:105FF000C89FF001C99FF00DD89FF00D1124E558FE
:10600000F14F8285882321F08181882309F087C0A0
:10601000EE2091F485E190E0C89FF001C99FF00D5A
:10602000D89FF00D1124E558F14F128A81858823FD
:1060300009F075C0178273C0133059F481E091E004
:10604000909393058093920581E0809391050F2DA5
:1060500008C0812F60E00E941F34812F6F2D0E94A5
:1060600000340F3799F485E190E0C89FF001C99F93
:10607000F00DD89FF00D1124E558F14F8091D40E0A
:10608000868785ED9EE0948B838B30C089E0089FE6
:10609000C0011124E091D10EF091D20EE80FF91F4A
:1060A0003396459154914115510571F485E190E085
:1060B000C89FF001C99FF00DD89FF00D1124E5583D
:1060C000F14F148A138A12C0FA01249185E190E0FD
:1060D000C89FF001C99FF00DD89FF00D1124E5581D
:1060E000F14F26874F5F5F4F548B438B85E190E0E4
:1060F000C89FF001C99FF00DD89FF00D1124E558FD
:10610000F14F17861186038711828FEF8087E78210
:10611000F282108A81E08287128A118A1482DF91CA
:10612000CF911F910F91FF90EF900895CF92DF9242
:10613000FF920F931F93CF93DF939091830E8091E3
:10614000840E282F30E0290F311D2F3F310519F023
:1061500014F02FEF30E02093830E9091980E8091F1
:10616000990E282F30E0290F311D2F3F310519F0EE
:1061700014F02FEF30E02093980E9091AE0E8091A6
:10618000AD0E282F30E0290F311D2F3F310519F0BA
:1061900014F02FEF30E02093AD0E9091C30E80915C
:1061A000C20E282F30E0290F311D2F3F310519F085
:1061B00014F02FEF30E02093C20E8091600388230B
:1061C00009F01AC136C1E091DA0EF091DB0E9F01A1
:1061D0002F5F3F4F3093DB0E2093DA0E44914F3FF9
:1061E00069F5A9014F5F5F4F5093DB0E4093DA0EC4
:1061F000F90184918F3219F4109260030BC186303B
:1062000009F0EBC0FA013196CF0101969093DB0EB5
:106210008093DA0EE491E33529F49093DE0E8093B7
:10622000DD0EDBC0E53409F0D8C08091DD0E909121
:10623000DE0E9093DB0E8093DA0ECFC047FF02C0D4
:106240004093D30E542F5F70842F90E0807F907026
:10625000803B910531F1803C910581F180399105B8
:1062600009F043C0C9010196F90144910196909348
:10627000DB0E8093DA0E0197FC012491852F90E0CC
:106280008C9FF0018D9FF00D9C9FF00D1124E5581F
:10629000F14F8081882309F4A0C0220F852F6385E8
:1062A00053C0C9010196F901449101969093DB0E08
:1062B0008093DA0E0197FC01249153C02F5F3F4F6A
:1062C0003093DB0E2093DA0E21503040F9012491F7
:1062D000852F90E08C9FF0018D9FF00D9C9FF00D1D
:1062E0001124E558F14F238778C08091D30E582FA1
:1062F0005F7090E0807F9070803B910541F1803C21
:10630000910509F45EC08039910509F066C02F5FE0
:106310003F4F3093DB0E2093DA0E21503040F901CD
:106320002491852F90E08C9FD0018D9FB00D9C9F74
:10633000B00D1124A558B14F8C91882309F44DC09C
:10634000220F852F1B966C910E94EA2F46C02F5F6B
:106350003F4F3093DB0E2093DA0E21503040F9018D
:106360002491473071F4852F90E08C9FF0018D9F30
:10637000F00D9C9FF00D1124E558F14F220F26835C
:106380002CC04C3571F4852F90E08C9FF0018D9FCF
:10639000F00D9C9FF00D1124E558F14F220F24833E
:1063A0001CC04436D1F4852F90E08C9FF0018D9F66
:1063B000F00D9C9FF00D1124E558F14F220F25831D
:1063C0000CC0852F90E08C9FF0018D9FF00D9C9F5D
:1063D000F00D1124E558F14F43878AED9EE00E94AD
:1063E000BF2F969587959093D90E8093D80E1092D3
:1063F000D00E1092CF0E02C0C5E1D0E06091CF0E5A
:106400007091D00E8091D80E9091D90E68177907AF
:1064100009F4D9CE6F5F7F4F7093D00E6093CF0E8B
:106420008091D50E9091D60E01969093D60E8093C2
:10643000D50E02E715E0CCE7DEE0FF24BFEFCB2E60
:10644000D12C8989882309F05EC08A899B89892B90
:1064500009F456C09E858D85981708F04CC050C031
:106460008A852A893B898F37E9F4D9018D91BB8BC5
:10647000AA8B8F3F01F1F90161811196BB8BAA8B29
:10648000E82FF0E0EE0FFF1FE05AF44F0190F0818B
:10649000E02D8F2D0995EA89FB8981918D87FB8BF2
:1064A000EA8B28C0A9014F5F5F4F5B8B4A8BF901D4
:1064B00084918F3F21F418821B8A1A8A21C04F5F72
:1064C0005F4F5B8B4A8B41505040FA01649190E0E2
:1064D000880F991F805A944FFC01259134918F2D7C
:1064E000F9010995EA89FB893196FB8BEA8B319793
:1064F000E491ED871E869E858D85981709F4B0CFAF
:106500008E858F5F8E878985882319F420E030E09F
:106510005DC08F858F3F11F08F5F8F879E8199239C
:1065200009F44EC02F81222309F44AC08D818823AB
:1065300009F446C04091D70E442309F441C0899F15
:10654000C001112480509F4F892F992730E0BC0152
:10655000629FC001639F900D729F900D1124805027
:106560009F4F892F9927242F30E0FC01E29FC00123
:10657000E39F900DF29F900D112480509F4F292F83
:1065800033278B818823F1F0EA81F0E0E050F54970
:10659000E491E058E89FC001112480509F4F892F5B
:1065A0009927A601481B590B429FC001439F900D9C
:1065B000529F900D112480509F4F292F332702C0E6
:1065C00020E030E08A819C81890F8A83F801208352
:1065D000F394065F1F4F6596F4E0FF1609F031CF84
:1065E000DF91CF911F910F91FF90DF90CF90089591
:1065F0001F93CF93DF93582F89E0589FC001112438
:106600002091D10E3091D20E280F391FC901039667
:10661000FC01A591B491F90184918150823010F46C
:1066200013E01DC08091910E8823B1F080919C0EE3
:10663000851711F4442381F48091A60E882371F00C
:106640008091B10E851711F4442341F49091A00E6E
:106650008091B50E891710F411E001C012E0212FCE
:1066600030E0FD01449185E190E0289FE001299F01
:10667000D00D389FD00D1124C558D14F4E8711969B
:10668000BC8BAB8B1F8680E58A836F838FEF8887F7
:1066900019861A8A188A21E02A87198A5C87298331
:1066A0001C82133049F481E091E09093930580932C
:1066B00092052093910508C0812F60E50E94003467
:1066C000812F69890E941F34DF91CF911F91089516
:1066D000FF920F931F93082FF62E0E94003410E0B4
:1066E00085E190E0089FF001099FF00D189FF00DE3
:1066F0001124E558F14FF2821F910F91FF900895F8
:10670000962F482F50E025E130E0429FF001439F53
:10671000F00D529FF00D1124E558F14F6281691B75
:1067200062830E9400340895482F50E025E130E054
:10673000429FF001439FF00D529FF00D1124E55848
:10674000F14F9281690F62830E9400340895000026
:106750000000000000000000000000000000000039
:106760000000000000000000000000000000000029
:106770000000000000000000000000000000000019
:106780000000000000000000000000000000000009
:1067900000000000000000000000000000000000F9
:1067A00000000000000000000000000000000000E9
:1067B00000000000000000000000000000000000D9
:1067C00000000000000000000000000000000000C9
:1067D00000000000000000000000000000000000B9
:1067E00000000000000000000000000000000000A9
:1067F0000000000000000000000000000000000099
:1068000099277727833008F00895E0E0F5E7660FD1
:10681000771FE60FF71FA591B491E2E7F5E02AE0B4
:10682000289FE00DF11DA183B2831124089590915A
:1068300091059170880F892B809391050895992770
:106840007727E2E7F5E02AE0289FE00DF11D6E3F93
:1068500031F4609191056E7F609391050BC06F3F9D
:1068600031F4609191056E6F6093910503C07BE6F2
:10687000760F75831124089599277727E2E7F5E0CD
:106880002AE0289FE00DF11D6083112408952F93C5
:106890003F934F935F936F937F938F939F93AF93A8
:1068A000BF93789411240E948C420E9458410E9408
:1068B00096302F923F924F925F926F927F928F927B
:1068C0009F92AF92BF92CF92DF92EF92FF920F937F
:1068D0001F93CF93DF9300906F05002019F4A1E67A
:1068E000B3E002C0A7E6B4E001E0002600926F0525
:1068F00002E00093700550919005609192057091AF
:106900009305809194052090730530907405409014
:10691000760550907705609075051091720570901E
:106920007D0580907E0590907F05A0908005B090B9
:10693000810520917C05C0908705D0908805E09066
:106940008A05F0908B0500918905309186059FEFAF
:10695000620C431CF2014491410300240008C12D44
:10696000D02D970CA81CF501449142030024000887
:10697000C10DD01D0C0DED1CF70144914303002403
:106980000008C10DD01D8A956AF440919105842FAD
:106990008695062E0694062600FA7695679576F972
:1069A00040FF66F940E860FD4FE74503002400081A
:1069B000C10DD01D0024C038D0050CF0CFE70A94DB
:1069C000C038D0050CF4C0E8C058CD939A9509F0B2
:1069D000BFCF409170054A954093700597E009F04C
:1069E000B7CF609275054092760590927F05A09290
:1069F000800500938905E0928A0560939205709363
:106A0000930580939405DF91CF911F910F91FF9093
:106A1000EF90DF90CF90BF90AF909F908F907F903E
:106A20006F905F904F903F902F9099278091280E04
:106A300077276091290E11240E94E62FBF91AF9114
:106A40009F918F917F916F915F914F913F912F9186
:106A500008950C942B350C942D350F931F932ABD5C
:106A6000E0916D05F0916E05019100000093B30077
:106A700005E0ED36F00710F40000000010F0E1E64C
:106A8000F3E0E0936D05F0936E05C895C895C89541
:106A9000C895C895C8950000000000002AB51F9150
:106AA0000F9108950000E091290EE0FFD6CFE1E1BB
:106AB000EA95F1F7000000000895000000000000D2
:106AC00000000000000000000000000000000000C6
:106AD00000000000000000000000000000000000B6
:106AE00000000000000000000000000000000000A6
:106AF0000000000000000000000000000000000096
:106B0000000306090C101316191C1F2225282B2E12
:106B1000313336393C3F414447494C4E5153555827
:106B20005A5C5E60626466686A6B6D6F70717374E4
:106B3000757678797A7A7B7C7D7D7E7E7E7F7F7F9D
:106B40007F7F7F7F7E7E7E7D7D7C7B7A7A79787683
:106B500075747371706F6D6B6A68666462605E5C99
:106B60005A585553514E4C494744413F3C393633AE
:106B7000312E2B2825221F1C191613100C09060371
:106B800000FDFAF7F4F0EDEAE7E4E1DEDBD8D5D278
:106B9000CFCDCAC7C4C1BFBCB9B7B4B2AFADABA843
:106BA000A6A4A2A09E9C9A9896959391908F8D8C66
:106BB0008B8A88878686858483838282828181818D
:106BC0008181818182828283838485868687888A87
:106BD0008B8C8D8F9091939596989A9C9EA0A2A451
:106BE000A6A8ABADAFB2B4B7B9BCBFC1C4C7CACD1C
:106BF000CFD2D5D8DBDEE1E4E7EAEDF0F4F7FAFD39
:106C0000808182838485868788898A8B8C8D8E8F0C
:106C1000909192939495969798999A9B9C9D9E9FFC
:106C2000A0A1A2A3A4A5A6A7A8A9AAABACADAEAFEC
:106C3000B0B1B2B3B4B5B6B7B8B9BABBBCBDBEBFDC
:106C4000C0C1C2C3C4C5C6C7C8C9CACBCCCDCECFCC
:106C5000D0D1D2D3D4D5D6D7D8D9DADBDCDDDEDFBC
:106C6000E0E1E2E3E4E5E6E7E8E9EAEBECEDEEEFAC
:106C7000F0F1F2F3F4F5F6F7F8F9FAFBFCFDFEFF9C
:106C8000000102030405060708090A0B0C0D0E0F8C
:106C9000101112131415161718191A1B1C1D1E1F7C
:106CA000202122232425262728292A2B2C2D2E2F6C
:106CB000303132333435363738393A3B3C3D3E3F5C
:106CC000404142434445464748494A4B4C4D4E4F4C
:106CD000505152535455565758595A5B5C5D5E5F3C
:106CE000606162636465666768696A6B6C6D6E6F2C
:106CF000707172737475767778797A7B7C7D7E7F1C
:106D000000020406080A0C0E10121416181A1C1E93
:106D100020222426282A2C2E30323436383A3C3E83
:106D200040424446484A4C4E50525456585A5C5E73
:106D300060626466686A6C6E70727476787A7C7E63
:106D40007F7D7B79777573716F6D6B696765636143
:106D50005F5D5B59575553514F4D4B494745434133
:106D60003F3D3B39373533312F2D2B292725232123
:106D70001F1D1B19171513110F0D0B090705030113
:106D8000FFFDFBF9F7F5F3F1EFEDEBE9E7E5E3E103
:106D9000DFDDDBD9D7D5D3D1CFCDCBC9C7C5C3C1F3
:106DA000BFBDBBB9B7B5B3B1AFADABA9A7A5A3A1E3
:106DB0009F9D9B99979593918F8D8B8987858381D3
:106DC00080828486888A8C8E90929496989A9C9ED3
:106DD000A0A2A4A6A8AAACAEB0B2B4B6B8BABCBEC3
:106DE000C0C2C4C6C8CACCCED0D2D4D6D8DADCDEB3
:106DF000E0E2E4E6E8EAECEEF0F2F4F6F8FAFCFEA3
:106E00007F7F7F7F7F7F7F7F7F7F7F7F7F7F7F7F92
:106E10007F7F7F7F7F7F7F7F7F7F7F7F7F7F7F7F82
:106E20007F7F7F7F7F7F7F7F7F7F7F7F7F7F7F7F72
:106E30007F7F7F7F7F7F7F7F7F7F7F7F7F7F7F7F62
:107100000309131E28313A40464C5054585B5E61C7
:10711000636567696B6C6E6F707172737475767787
:10712000777879797A7A7B7B7C7C7C7D7D7D7E7EAD
:107130007E7E7F7F7F7F7F7F7F7F7F7F7F7F7F7F61
:107140007F7F7F7F7F7F7F7F7F7F7F7F7F7E7E7E52
:107150007E7D7D7D7C7C7C7B7B7A7A797978777784
:10716000767574737271706F6E6C6B69676563614D
:107170005E5B5854504C46403A31281E13090300B8
:10718000C6CCD5DBDFE3E5E7E9EAEBECEDEEEFEFCC
:10719000F0F0F0F1F1F1F1F2F2F2F2F2F2F2F2F3D8
:1071A000F3F3F3F3F3F3F3F3F3F3F3F3F3F3F3F3AF
:1071B000F3F3F3F3F3F3F3F3F3F3F3F3F3F3F3F39F
:1071C000F3F3F3F3F3F3F3F3F3F3F3F3F3F3F3F38F
:1071D000F3F3F3F3F3F3F3F3F3F3F3F3F3F3F3F37F
:1071E000F2F2F2F2F2F2F2F2F1F1F1F1F0F0F0EF8C
:1071F000EFEEEDECEBEAE9E7E5E3DFDBD5CCC6004B
:1072000000283D42302D2C2B2C2D2E2F30323335A3
:1072100037393B3D3F414345484A4C4E5053555703
:10722000595B5D5F61636567696B6C6E70717374E8
:10723000757778797A7B7C7D7D7E7E7F7F7F7F7F8F
:107240007F7F7F7F7F7F7E7E7D7D7C7B7A79787775
:1072500075747371706E6C6B69676563615F5D5B9C
:1072600059575553504E4C4A484543413F3D3B3991
:1072700037353332302F2E2D2C2B2C2D30423D28FC
:1072800000E9E5FED4D7D7D7D6D4D2D0CECCCAC861
:10729000C6C3C1BFBDBAB8B6B4B1AFADABA9A7A59F
:1072A000A3A19F9E9C9A999795949391908F8D8C72
:1072B0008B8A898888878685858484848383838371
:1072C0008383838383848484858586878888898A69
:1072D0008B8C8D8F909193949597999A9C9E9FA15A
:1072E000A3A5A7A9ABADAFB1B4B6B8BABDBFC1C372
:1072F000C6C8CACCCED0D2D4D6D7D7D7D4FEE5E92B
:10730000F9F8F9F5EBE1DDDEE0E2E4E5E6E5E4E2FB
:10731000DED9D2CAC1B7ACA299918A868381808016
:107320008182838586888A8C8D8F9092939596979B
:1073300098999A9B9B9C9D9D9D9E9E9E9F9F9F9F83
:107340009F9F9F9E9E9E9D9D9D9C9B9B9A9998977B
:1073500096959392908F8D8C8A8886858382818082
:10736000808183868A9199A2ACB7C1CAD2D9DEE264
:10737000E4E5E6E5E4E2E0DEDDE1EBF5F9F8F9006D
:107380000708070B151F2322201E1C1B1A1B1C1E7F
:1073900022272E363F49545E676F767A7E7F7F7F45
:1073A0007F7E7D7B7A7876747371706E6D6B6A699F
:1073B0006867666565646463636262626161616196
:1073C000616161626262636363646565666768697F
:1073D0006A6B6D6E7071737476787A7B7D7E7F7F59
:1073E0007F7F7E7A766F675E54493F362E27221E56
:1073F0001C1B1A1B1C1E2022231F150B070807002D
:107400001F313D444E5354565A5F64696E74767909
:107410007C7F7F7F7F7F7F7F7F7F7F7F7F7F7F7F7F
:107420007F7F7F7F7F7F7F7F7F7F7F7F7F7F7F7F6C
:107430007F7F7F7F7F7F7F7F7F7F7F7F7F7F7F7F5C
:107440007F7F7F7F7F7F7F7F7F7F7F7F7F7F7F7F4C
:107450007F7F7F7F7F7F7F7F7F7F7F7F7F7F7F7F3C
:107460007F7F7F7F7F7F7F7F7F7F7F7F7F7F7F7F2C
:107470007F7F7F7F7F7F7F7F7F7F7F7C7871684C7E
:107480002C1C120C0A0B0A05FDF3E9DFD4CAC0B7A5
:10749000AEA69E97918B868582808080808080803A
:1074A00080808080808080808080808080808080DC
:1074B00080808080808080808080808080808080CC
:1074C00080808080808080808080808080808080BC
:1074D00080808080808080808080808080808080AC
:1074E000808080808080808080808080808080809C
:1074F000808080808087919DACC4CBD4DDF2FAFA85
:1075000022002400260028002B002D00300033002C
:10751000360039003D004000440048004C00510056
:1075200056005B00600066006C007300790081000B
:10753000880090009900A200AC00B600C100CC0009
:10754000D800E500F30001011001210132014401DE
:1075500057016C0181019801B001CA01E5010202E5
:107560002102410264028802AE02D7020303300303
:1075700061039403CB03050442048304C70410058C
:107580005D05AF0505066106C206290796070908CD
:10759000830805098E09200ABA0A5D0B0A0CC10C82
:1075A000840D510E2B0F121007110A121D134014D7
:1075B0007415BA1614188319071BA31C571E242010
:1075C0000E22142439267F28E82A752D2930063307
:1075D0000F364539AD3C49401B442848734CFE509A
:1075E000CF55EA5A51600C661D6C8B725A799280A5
:1075F00037885090E598FDA19FABD3B5A3C000009C
:107600001F93CF93DF93FA01549131961491C52FB4
:10761000D0E09F012F5F3F4F70E095E0660F771F2E
:107620009A95E1F7680F711D40E00BC084918D932E
:107630009F5F31969517D0F34F5F2C0F3D1F605E13
:107640007F4F411730F4DB01A056BA4FF90190E0AB
:10765000F1CFDF91CF911F910895382F603CD0F486
:1076600070E0660F771FCB018A58944FFC0124917C
:107670006958744FFB016491832F90E0FC0174E022
:10768000EE0FFF1F7A95E1F7E81BF90BE050F64F7C
:1076900021876287832F90E0FC0154E0EE0FFF1FEB
:1076A0005A95E1F7E81BF90BE050F64F81852381ED
:1076B0003481280F311D3687258746954695469596
:1076C000842F90E045E0880F991F4A95E1F7280F35
:1076D000391F3487238708950F931F93CF93DF9328
:1076E0008C01C0E0D0E007C00E944B438823E1F347
:1076F0000E944E432196C017D107B4F3DF91CF917A
:107700001F910F91089540520E9472420895FF9276
:107710000F931F93CF93DF938C01F62EEA01FE01A6
:1077200044912196442349F0802F0F5F1F4F4F77DC
:1077300040526F2D0E947242F2CFDF91CF911F9184
:107740000F91FF900895FF920F931F93CF93DF93B4
:10775000EC01F62E142F00E0112311F4002361F444
:107760002C2F2197812F6AE00E94BF5A905F822FB1
:107770006F2D492F0E9472420F5F033031F0812F2D
:107780006AE00E94BF5A182FE7CFDF91CF911F9177
:107790000F91FF900895CF92DF92EF92FF920F9397
:1077A0001F93CF93DF93C62E79018A01EC01DD246C
:1077B000E114F1040105110511F4DD2069F4C8019B
:1077C000B7012AE030E040E050E00E94F25A462F34
:1077D000405F8C2F6C2D03C08C2F6C2D40E00E94DD
:1077E0007242D394219786E0D81669F0C801B70198
:1077F0002AE030E040E050E00E94F25AC901DA018C
:107800007C018D01D5CFDF91CF911F910F91FF901A
:10781000EF90DF90CF9008957F928F929F92AF92DA
:10782000BF92CF92DF92EF92FF920F931F93CF936D
:10783000DF93782E862EEA01FA01C590D490FA01E2
:107840003296A590B49000E016C0FC01EE0DFF1D2D
:107850003296EE0FFF1FEC0FFD1F45915491812FC3
:10786000870D692D0E9464421F5F812F90E08C1567
:107870009D055CF30F5F802F90E08A159B055CF4FB
:107880008C9D70018D9DF00C9C9DF00C112410E0DE
:10789000902E980CEACFDF91CF911F910F91FF901E
:1078A000EF90DF90CF90BF90AF909F908F907F90A0
:1078B00008951842224230424641EBEDC89500003F
:1078C000EA95E1F700C000C04091050A5091060A10
:1078D0004ABD5BBDC0910B0AD0910C0A40900D0AC5
:1078E00050900E0A9090070AF090020AE0900A0A5F
:1078F0007091010A672F6770882400EDA02EA2E125
:10790000BAE075D00027E101D30108B9F1E0E091B8
:10791000220E119311931193119311931193E091EE
:10792000230E119311931193119311931193E091DD
:10793000240E119311931193119311931193E091CC
:10794000250E119311931193119311931193E091BB
:10795000260E119311931193119311931193639523
:107960007395FA94A9F483940FE0809EF001E0509F
:10797000F64F058016800ABC1BBCC385D4854584A0
:1079800056849780F280E2847181672F677008C007
:107990000000000000000000000009E00A95F1F777
:1079A000791509F4E20109F4772709F46627AA9406
:1079B00041F0683019F000C000C0A3CF6627A09640
:1079C000A0CFC895C8950E9409424091290E405DFC
:1079D0004093290E11E000912B0E012700932B0EEE
:1079E000E1E0E0932A0EE2E0E09336000895289863
:1079F000E0916D05F0916E05019125E0ED36F207FD
:107A000021E633E00093B30008F0F901E0936D053F
:107A1000F0936E051E01C090100AD090110A80E309
:107A200023E036E0D1E040EA59E098E00D91099F6B
:107A3000112D0F71FA01029FE00DF11D0281C0812D
:107A4000F601089FE00DF11D139FE00DF11DC0939D
:107A5000220E0590099205900992059009920590D1
:107A6000099205900992059009920D91099F112D97
:107A70000F71FA01029FE00DF11D0281C081F60134
:107A8000089FE00DF11D139FE00DF11DC093230E23
:107A90000590099205900992059009920590099226
:107AA0000D91289A0590099205900992099F112D30
:107AB0000F71FA01029FE00DF11D0281C081F601F4
:107AC000089FE00DF11D139FE00DF11DC093240EE2
:107AD00005900992059009920590099205900992E6
:107AE00005900992059009920D91099F112D0F7132
:107AF000FA01029FE00DF11D0281C081F601089F8D
:107B0000E00DF11D139FE00DF11DC093250E0590B2
:107B100009920590099205900992059009920590A5
:107B20000992059009920D91099F112D0F71FA018B
:107B3000029FE00DF11D0281C081F601089FE00D5A
:107B4000F11D139FE00DF11DC093260E05900992C3
:107B50000590099205900992059009920590099265
:107B600005900992E1013D01DE011EEF4AB55BB5CA
:107B7000639FC0013A2F307ECE2DCC0FDD27C0573A
:107B8000DE4FE991F881C6E0D1E0CC9020E3C29EBF
:107B9000A395AF71A32B040E151E080E191E099490
:107BA000F001C895C895C895C8950591D990D1128E
:107BB0000D2D08B9CC900591D990D1120D2D08B991
:107BC000C29E0591D990D1120D2D08B9040E151E33
:107BD0000591D990D1120D2D08B9080E191E0591E5
:107BE000D990D1120D2D08B9A395AF710591D990F7
:107BF000D1120D2D08B9A32BF0010591D990D11206
:107C00000D2D08B9CC900591D990D1120D2D08B940
:107C1000C29E0591D990D1120D2D08B9040E151EE2
:107C20000591D990D1120D2D08B9080E191E059194
:107C3000D990D1120D2D08B9A395AF710591D990A6
:107C4000D1120D2D08B9A32BF0010591D990D112B5
:107C50000D2D08B9CC900591D990D1120D2D08B9F0
:107C6000C29E0591D990D1120D2D08B9040E151E92
:107C70000591D990D1120D2D08B9080E191E059144
:107C8000D990D1120D2D08B9A395AF710591D99056
:107C9000D1120D2D08B9A32BF0010591D990D11265
:107CA0000D2D08B9CC900591D990D1120D2D08B9A0
:107CB000C29E0591D990D1120D2D08B9040E151E42
:107CC0000591D990D1120D2D08B9080E191E0591F4
:107CD000D990D1120D2D08B9A395AF710591D99006
:107CE000D1120D2D08B9A32BF0010591D990D11215
:107CF0000D2D08B9CC900591D990D1120D2D08B950
:107D0000C29E0591D990D1120D2D08B9040E151EF1
:107D10000591D990D1120D2D08B9080E191E0591A3
:107D2000D990D1120D2D08B9A395AF710591D990B5
:107D3000D1120D2D08B9A32BF0010591D990D112C4
:107D40000D2D08B9CC900591D990D1120D2D08B9FF
:107D5000C29E0591D990D1120D2D08B9040E151EA1
:107D60000591D990D1120D2D08B9080E191E059153
:107D7000D990D1120D2D08B9A395AF710591D99065
:107D8000D1120D2D08B9A32BF0010591D990D11274
:107D90000D2D08B9CC900591D990D1120D2D08B9AF
:107DA000C29E0591D990D1120D2D08B9040E151E51
:107DB0000591D990D1120D2D08B9080E191E059103
:107DC000D990D1120D2D08B9A395AF710591D99015
:107DD000D1120D2D08B9A32BF0010591D990D11224
:107DE0000D2D08B9CC900591D990D1120D2D08B95F
:107DF000C29E0591D990D1120D2D08B9040E151E01
:107E00000591D990D1120D2D08B9080E191E0591B2
:107E1000D990D1120D2D08B9A395AF710591D990C4
:107E2000D1120D2D08B9A32BF0010591D990D112D3
:107E30000D2D08B9CC900591D990D1120D2D08B90E
:107E4000C29E0591D990D1120D2D08B9040E151EB0
:107E50000591D990D1120D2D08B9080E191E059162
:107E6000D990D1120D2D08B9A395AF710591D99074
:107E7000D1120D2D08B9A32BF0010591D990D11283
:107E80000D2D08B9CC900591D990D1120D2D08B9BE
:107E9000C29E0591D990D1120D2D08B9040E151E60
:107EA0000591D990D1120D2D08B9080E191E059112
:107EB000D990D1120D2D08B9A395AF710591D99024
:107EC000D1120D2D08B9A32BF0010591D990D11233
:107ED0000D2D08B9CC900591D990D1120D2D08B96E
:107EE000C29E0591D990D1120D2D08B9040E151E10
:107EF0000591D990D1120D2D08B9080E191E0591C2
:107F0000D990D1120D2D08B9A395AF710591D990D3
:107F1000D1120D2D08B9A32BF0010591D990D112E2
:107F20000D2D08B9CC900591D990D1120D2D08B91D
:107F3000C29E0591D990D1120D2D08B9040E151EBF
:107F40000591D990D1120D2D08B9080E191E059171
:107F5000D990D1120D2D08B9A395AF710591D99083
:107F6000D1120D2D08B9A32BF0010591D990D11292
:107F70000D2D08B9CC900591D990D1120D2D08B9CD
:107F8000C29E0591D990D1120D2D08B9040E151E6F
:107F90000591D990D1120D2D08B9080E191E059121
:107FA000D990D1120D2D08B9A395AF710591D99033
:107FB000D1120D2D08B9A32BF0010591D990D11242
:107FC0000D2D08B9CC900591D990D1120D2D08B97D
:107FD000C29E0591D990D1120D2D08B9040E151E1F
:107FE0000591D990D1120D2D08B9080E191E0591D1
:107FF000D990D1120D2D08B9A395AF710591D990E3
:10800000D1120D2D08B9A32BF0010591D990D112F1
:108010000D2D08B9CC900591D990D1120D2D08B92C
:10802000C29E0591D990D1120D2D08B9040E151ECE
:108030000591D990D1120D2D08B9080E191E059180
:10804000D990D1120D2D08B9A395AF710591D99092
:10805000D1120D2D08B9A32BF0010591D990D112A1
:108060000D2D08B9CC900591D990D1120D2D08B9DC
:10807000C29E0591D990D1120D2D08B9040E151E7E
:108080000591D990D1120D2D08B9080E191E059130
:10809000D990D1120D2D08B9A395AF710591D99042
:1080A000D1120D2D08B9A32BF0010591D990D11251
:1080B0000D2D08B9CC900591D990D1120D2D08B98C
:1080C000C29E0591D990D1120D2D08B9040E151E2E
:1080D0000591D990D1120D2D08B9080E191E0591E0
:1080E000D990D1120D2D08B9A395AF710591D990F2
:1080F000D1120D2D08B9A32BF0010591D990D11201
:108100000D2D08B9CC900591D990D1120D2D08B93B
:10811000C29E0591D990D1120D2D08B9040E151EDD
:108120000591D990D1120D2D08B9080E191E05918F
:10813000D990D1120D2D08B9A395AF710591D990A1
:10814000D1120D2D08B9A32BF0010591D990D112B0
:108150000D2D08B9CC900591D990D1120D2D08B9EB
:10816000C29E0591D990D1120D2D08B9040E151E8D
:108170000591D990D1120D2D08B9080E191E05913F
:10818000D990D1120D2D08B9A395AF710591D99051
:10819000D1120D2D08B9A32BF0010591D990D11260
:1081A0000D2D08B9CC900591D990D1120D2D08B99B
:1081B000C29E0591D990D1120D2D08B9040E151E3D
:1081C0000591D990D1120D2D08B9080E191E0591EF
:1081D000D990D1120D2D08B9A395AF710591D99001
:1081E000D1120D2D08B9A32BF0010591D990D11210
:1081F0000D2D08B9CC900591D990D1120D2D08B94B
:10820000C29E0591D990D1120D2D08B9040E151EEC
:108210000591D990D1120D2D08B9080E191E05919E
:10822000D990D1120D2D08B9A395AF710591D990B0
:10823000D1120D2D08B9A32BF0010591D990D112BF
:108240000D2D08B9CC900591D990D1120D2D08B9FA
:10825000C29E0591D990D1120D2D08B9040E151E9C
:108260000591D990D1120D2D08B9080E191E05914E
:10827000D990D1120D2D08B9A395AF710591D99060
:10828000D1120D2D08B9A32BF001089528980E9452
:108290002935E7E1EA95F1F7289A05D1E0E0F6E023
:1082A000E8D0E0FF43D0E0FF02C00E9447340895C9
:1082B000129A0C945B410C945D4112984427552707
:1082C000662777278CE00C9465410C9467410C94E9
:1082D00069410C946B410C946D410C946F41440FB7
:1082E000551F00994160660F771F01996160139ACD
:1082F0000C947A410C947C4113980C947F410C941B
:1083000081410C9483410C9485418A9541F74095B5
:108310005095609570955F707F7040932F0E5093CD
:10832000300E6093310E7093320E0895EF93E0910A
:10833000290EE53EE0F5E531D0F12F923F924F92C4
:108340005F926F927F928F929F92AF92BF92CF92E5
:10835000DF92EF92FF920F931F932F933F934F93D0
:108360005F936F937F938F939F93AF93BF93CF93BD
:10837000DF930E945D3CDF91CF91BF91AF919F91C0
:108380008F917F916F915F914F913F912F911F91AD
:108390000F91FF90EF90DF90CF90BF90AF909F90A4
:1083A0008F907F906F905F904F903F902F90EF91C4
:1083B0000895FF93EF93EFB7EF93E0918400EE50B1
:1083C000E13000F0E23000F0E33000F0E43000F0A3
:1083D000E53000F0E63000F0E73000F0E83000F083
:1083E000E93000F005D0EF91EFBFEF91FF911895C4
:1083F0000F921F92E2EBF8E70090280E000C112478
:10840000E00DF11D05901490F00109951F900F905B
:10841000089528980E942935E5E1EA95F1F7E09161
:10842000290EEA95E093290E289A0000000008958D
:1084300028980E945235289A0000E1E0F6E019D011
:108440002BD0089528980E945235E0EB0000EA9561
:10845000E9F700000000289AF6E0E2E00AD008956B
:1084600028980E945235289A0000E3E0FDEF01D0E1
:1084700008950090290E0A9410905F0011FC0F2EB1
:108480000092290E0090280E11FC0E2E0092280E4C
:10849000E0E011FCE1E00895E3E0E0938900EDE81D
:1084A000E09388000895E7E0E0938900EBE1E09332
:1084B00088000895E0E0F4E0A0EAB5E066276D9357
:1084C0003197E9F7112408959927772720E2629FD1
:1084D000080E191EA0EAB5E0A00DB11D4C931124A1
:1084E00008950895992720E2629F080E191EA0EAB8
:1084F000B5E0A00DB11D50912E0E450F4C931124E7
:10850000089580932E0E089580930F0A0895809306
:10851000100A9093110A0895EF92FF920F931F9300
:10852000CF93DF93E0E0FAE020E0822F6081418189
:10853000EF93FF932F930E942D3B2F91FF91EF918B
:108540003F962395213088F3552721E0662775E073
:1085500082E19AE0E0E0FAE030854281EC01579F49
:10856000C00DD11D540F442349F0317039F0699387
:1085700069936993699369934A95C9F73F962A95D8
:1085800059F731E020910F0A213011F43091270E74
:1085900000EA19E0780123E0A5E0B0E241E0F7014C
:1085A000329FE00DF11D008111811030E9F1183D7D
:1085B000D8F50030C9F10A38B8F560E0712F760FB0
:1085C000783068F1783D58F57850EC017A9FC00D0D
:1085D000D11D0880002021F46B9F030E08821FC06C
:1085E0000980002021F46B9F030E098218C00A80C5
:1085F000002021F46B9F030E0A8211C00B80002023
:1086000021F46B9F030E0B820AC00C80002039F40A
:108610006B9F030E0C82032E0A940092270E259660
:1086200073956395683050F23395303208F031E03D
:108630004395403208F4B3CF7091270E703208F0A2
:1086400071E07093270E552721E0662775E0E0E082
:10865000FAE030854281EC01579FC00DD11D540FC7
:10866000442349F0317039F46993699369936993AC
:1086700069934A95C9F73F962A9559F71124DF91D6
:10868000CF911F910F91FF90EF90089580932C0E42
:1086900090932D0E089580912A0E08951124109222
:1086A0002A0E0895882329F480912F0E9091300E80
:1086B00008958091310E9091320E089580E891E0F6
:1086C0008093610090936100089580E890E080932A
:1086D00061009093610008959091620E992311F4C6
:1086E00086E005C086E0989FC00111248F538093D7
:1086F00099019091630E992319F41092640E0895D4
:1087000086E0989FC001112485548093640E0895DB
:1087100070E025E130E0629FF001639FF00D729FF1
:10872000F00D1124E80FF11DE356FE4F80810895EE
:10873000A82FB0E0FD01E250F14F8081813059F067
:10874000823039F4FD01E151F14F4081A450B14F25
:1087500013C0833049F4FD01E151F14F4081A45031
:10876000B14F8C91861B0AC0FD01E151F14FA4501D
:10877000B14F843099F440818C91860F90E025E1CF
:1087800030E0829FF001839FF00D929FF00D112445
:10879000E40FF11DE356FE4F8081089540818C91D6
:1087A00090E025E130E0829FF001839FF00D929FE1
:1087B000F00D1124E40FF11DE356FE4F8081089562
:1087C00070E025E130E0629FF001639FF00D729F41
:1087D000F00D1124E80FF11DE356FE4F408308957C
:1087E00008951092030F1092020F1092FA0E109239
:1087F000F90EE82FF0E0E250F14FE081EE23E9F0CE
:10880000E13019F48FEF9FEF04C0E23039F481E0DA
:1088100090E09093030F8093020F0895E33039F4B2
:108820008FEF9FEF9093FA0E8093F90E089581E0F9
:1088300090E09093FA0E8093F90E08951092030F32
:108840001092020F1092FA0E1092F90E8823E9F09E
:10885000813019F48FEF9FEF04C0823039F481E04A
:1088600090E09093030F8093020F0895833039F4C2
:108870008FEF9FEF9093FA0E8093F90E089581E0A9
:1088800090E09093FA0E8093F90E08951F938091D3
:10889000DF0E6091E00E9091E30E30E0A5E1B0E0D4
:1088A00012E073E035C0822F90E08A9FF0018B9F29
:1088B000F00D9A9FF00D1124E40FF51FE356FE4FC3
:1088C000808160E08730A1F0883018F48630D9F4D8
:1088D00005C0883041F08930B1F410C03093EF0EFC
:1088E0002093FC0E09C03093EF0E2093FC0E0AC0BB
:1088F0003093F00E2093FD0E108305C03093F00EE0
:108900002093FD0E70832F5F243169F63F5F94E161
:10891000343120F420E0432F50E0F6CF8093DF0E77
:108920006093E00E9093E30E3093770E1F910895BD
:1089300090919401882359F0EEEFFEE0292F30E06A
:108940002E0F3F1F62E051E043E094E031C0EEEFB4
:10895000FEE0292F30E02E0F3F1F61E052E044E09F
:1089600093E011C08081813011F490830BC082307C
:1089700011F4408307C0833011F4508303C0843066
:1089800009F460833196E217F30761F70895808157
:10899000813011F490830BC0823011F4408307C002
:1089A000833011F4508303C0843009F4608331961E
:1089B000E217F30761F708952F923F924F925F926B
:1089C0006F927F928F929F92AF92BF92CF92DF92DF
:1089D000EF92FF920F931F93DF93CF93CDB7DEB744
:1089E000C159D1400FB6F894DEBF0FBECDBFCF56F0
:1089F000DE4F8883C159D1402090EF0E3090FC0E9D
:108A00001091E10E0091E20EF090ED0EE090EE0E6E
:108A1000D090DF0EA090E00E8091E30E70E065E153
:108A2000462E512C54E1652E712C4E010894811C68
:108A3000911C3BC0262F30E0CA01B42EC92E249DC4
:108A4000F001259DF00D349DF00D1124E40FF51F6C
:108A5000E356FE4FE081269DD001279DB00D369D47
:108A6000B00D1124A40FB51FA80DB91DEC93271646
:108A700069F4361659F4DE2EAA2483E0E81719F4B7
:108A800098E09C9309C086E08C9306C0B12EC02E5E
:108A90002F2D3E2DC9019C016F5F1B2D0C2DF22E39
:108AA000E32E643139F67F5F84E1743120F460E0B5
:108AB000472F50E0F6CF1093E10E0093E20EF092B4
:108AC000ED0EE092EE0ED092DF0EA092E00E8093BB
:108AD000E30E7093770ECF56DE4F9881C159D14087
:108AE0009923C9F520E004E110E045E1C42ED12C22
:108AF0007E010894E11CF11C1CC0F0E0C8018E1B33
:108B00009F0B8C9DD0018D9DB00D9C9DB00D1124AF
:108B1000A40FB51FA356BE4FE60FF71FEE0DFF1DA6
:108B200080818C93E32F3E2F3F5F353131F72F5FEC
:108B300084E1243158F4E0E0422F50E0409FB0013E
:108B4000419F700D509F700D1124EDCF8093E30E67
:108B50002093770E36C090E035E1C32ED12C24E16E
:108B6000E22EF12C8E010F5F1F4F1AC0F0E0EC9D3A
:108B7000D001ED9DB00DFC9DB00D1124A21BB30BD7
:108B8000A356BE4FE40FF51FE00FF11F80815496EE
:108B90008C93E62F6E2F6F5F653141F79F5F84E105
:108BA000943158F4E0E0292F30E02E9DA0012F9D54
:108BB000500D3E9D500D1124EDCF8093E30E909308
:108BC000770E8091650E8F5F8093650E843010F074
:108BD0001092650ECF56DE4F0FB6F894DEBF0FBE73
:108BE000CDBFCF91DF911F910F91FF90EF90DF905C
:108BF000CF90BF90AF909F908F907F906F905F903D
:108C00004F903F902F90089580916A0E882301F530
:108C10001092770E2091E30E30E0A5E1B0E020C085
:108C2000622F6F5F822F90E08A9FF0018B9FF00D83
:108C30009A9FF00D1124E40FF51FE356FE4F80813B
:108C4000833011F0262F09C02093E30E3093770E66
:108C500080E0089520E0432F50E0243109F73F5F82
:108C60003431C0F32093E30E3093770E81E080938C
:108C70006A0E1092510E1092500E089520916B0EB4
:108C800030E049EB51E0249FF001259FF00D349F27
:108C9000F00D1124E80FF11D85E1689FB00111244A
:108CA000E60FF71FE256F24BE4918E2F0895CF9214
:108CB000DF92EF92FF920F931F93CF93DF93C82F12
:108CC000D0E08E010151114FF8012081BCEFEB2E55
:108CD000BEE0FB2EEC0EFD1EF701808190E0A5E1C9
:108CE000CA2ED12C8C9DF0018D9DF00D9C9DF00D18
:108CF0001124E20FF11DE356FE4F808190E0909326
:108D0000E00E8093DF0E02970CF45AC0862F0E946B
:108D10001E44F80120814091F90E5091FA0EA22FC5
:108D2000A40FF70130816091020F7091030FB32FF0
:108D3000B60F8B2F90E08C9DF0018D9DF00D9C9DCA
:108D4000F00D1124EA0FF11DE356FE4FE081E09390
:108D5000DF0E1092E00EE43039F0E53018F4E23026
:108D600078F522C0E53061F5440F551F240F660FDA
:108D7000771F360F832F90E08C9DF0018D9DF00DB5
:108D80009C9DF00D1124E20FF11DE356FE4F8081F2
:108D900090E09093E00E8093DF0E0297FE01E75182
:108DA000F14F029718F0108280E00BC081E08083C1
:108DB000FE01EF50F14FA083CB50D14FB88301C0DB
:108DC00081E0DF91CF911F910F91FF90EF90DF90A5
:108DD000CF9008952F923F924F925F926F927F9221
:108DE0008F929F92AF92BF92CF92DF92EF92FF92BB
:108DF0000F931F93CF93DF931092770EB5E1AB2EB5
:108E0000B12CA3E02A2E312CF4E04F2E512CE5E0BA
:108E10006E2E712CF9C0822F90E0FC01E250F14FD0
:108E20003081332309F4EBC0FC01E950F14F80811C
:108E30008F5F8083333010F4883018F4863008F464
:108E4000DEC0822F0E94F1438091770EC82FD0E0C0
:108E5000FE01E751F14F8081882309F4A3C0FE0190
:108E6000E151F14F60814091F90E5091FA0E862E3A
:108E7000840EFE01E450F14F90812091020F309159
:108E8000030F992E920EE92CFF24C82CDD24EA9CB6
:108E9000F001EB9CF00DFA9CF00D1124EC0DFD1D82
:108EA000E356FE4F8081A82FB0E0B093E00EA09370
:108EB000DF0E220F331F920F092F10E0440F551FB2
:108EC000640F70E00A9DF0010B9DF00D1A9DF00DEE
:108ED0001124E60FF71FE356FE4F8081282F30E064
:108EE0003093EE0E2093ED0ECD010497029760F4BF
:108EF0002330310529F47092E00E6092DF0E04C039
:108F00005092E00E4092DF0E159729F43092E20E57
:108F10002092E10E06C022E030E03093E20E209372
:108F2000E10E0A9DF0010B9DF00D1A9DF00D11242C
:108F3000E60FF71FE356FE4F8091DF0E808380918E
:108F4000E10EEA9CD001EB9CB00DFA9CB00D11240F
:108F5000AC0DBD1DA356BE4F8C938230D1F48091D1
:108F60006B0E90E029EB31E0829FF001839FF00DC2
:108F7000929FF00D1124E80DF11D35E1939EC00183
:108F80001124E80FF91FE256F24B8491833009F463
:108F90008C938091660E9091670E01969093670E68
:108FA0008093660EFE01E151F14F80819091F90EA0
:108FB000890F8083FE01E450F14F80819091020F70
:108FC000890F8083FE01E250F14F1082FE01E950CB
:108FD000F14F1082FE01EF50F14F8AEF8083FE01C6
:108FE000EB50F14F80838091680E9091690E01964D
:108FF0009093690E8093680EC751D14F188280916B
:10900000770E8F5F8093770E2091770E8091940179
:10901000281708F400CFDF91CF911F910F91FF9097
:10902000EF90DF90CF90BF90AF909F908F907F9008
:109030006F905F904F903F902F900895E62FF0E053
:1090400095E0EE0FFF1F9A95E1F7E80FF11DE0564E
:10905000FA4F8091640E840F80830895E62FF0E02C
:1090600025E0EE0FFF1F2A95E1F7E80FF11DE0560E
:10907000FA4F408308958FEF8093A4098093A70946
:109080008093AA098093AD090895089508950E94D8
:109090005A4280E00E94844284E190E00E94B45AE7
:1090A00010926B0E80E00E94524381E00E94524376
:1090B0001092430E1092420E1092410E1092400EEA
:1090C00081E08093610E8093490E89E996E40E94C5
:1090D000672F80EB97E40E94812F87E00E948142F6
:1090E000089510925A0E81E080935B0E84E190E027
:1090F0000E946C3B089591E09093490E8093580E26
:109100001092710E1092590E9093610E90939501EA
:1091100081E090E00E946C3B80EB97E40E94812FFD
:1091200008950F931F93CF93DF939091940180E064
:109130001AC0E82FF0E0DF01AB50B14F1C92DF0105
:10914000AF50B14F1C92DF01A250B14F1C92DF0112
:10915000A950B14F1C92DF01A450B14F1C92E151B4
:10916000F14F10828F5F891720F32091920130E038
:1091700080916B0E90E08217930714F010926B0EA3
:109180008091710E4091E30E8823C1F580916B0EA2
:1091900090E029EB31E0829FE001839FD00D929F08
:1091A000D00D1124842F40E055E105E110E023C0EB
:1091B000459F900111242C0F3D1FA0E0842F90E0CB
:1091C000809FB001819F700D909F700D11240DC084
:1091D000B0E0FD01E20FF31FE256F24BE491A60F5F
:1091E000B71FA356BE4FEC93A82F8A2F8F5F8531F0
:1091F00079F74F5F84E14431D8F20DC0842F90E0BD
:1092000006C000008F5F8531E1F79F5F84E19431F4
:1092100010F480E0F7CF8093E30E30916A0E8091D6
:10922000680E9091690E4091660E5091670E20E095
:1092300017C0A22FB0E0FD01E751F14F1082FD01F0
:10924000E250F14F1082FD01EB50F14F1082AF5010
:10925000B14F1C922F5F40E050E080E090E030E0A2
:10926000223038F330936A0E9093690E8093680E23
:109270005093670E4093660E2093770E8FEF809386
:10928000A4098093A7098093AA098093AD090E943D
:1092900046448091650E8F5F8093650E843010F098
:1092A0001092650E81E090E00E946C3BDF91CF91BF
:1092B0001F910F9108958091770EA82FB0E0FD01C6
:1092C000E151F14F8081843128F4A450B14F8C9149
:1092D000843110F00E94914808951F938091950168
:1092E0008823B1F11092950110926A0E1092760EB9
:1092F0001092750E10924A0E80916B0E8093720E32
:1093000080914F0E482F50E082E08093490E20E07C
:1093100030E008C02F5F3F4F849131968F3FD1F7E7
:1093200041505040F901EC50F84A4115510591F770
:109330001092740E1092730E2F5F3F4F30934D0EAC
:1093400020934C0E849180936B0E0E94914898C09C
:109350008091400E9091410E90FF06C08091440E86
:109360009091450E90FF75C08091F70E882309F00B
:1093700087C080914A0E823020F0815080934A0E3F
:1093800039C0E0914C0EF0914D0E9F012F5F3F4F81
:1093900030934D0E20934C0EEC50F84A6491462FBA
:1093A00050E05093740E4093730E4031510520F0FD
:1093B000CA0141970F9798F460934A0E2F5F3F4F71
:1093C00030934D0E20934C0E215030402C50384A93
:1093D000F90184918093750E1092760E04C050931B
:1093E000760E4093750E8091750E9091760E8F3F9C
:1093F000910579F11091750E17FF08C080E061E0CA
:109400000E945746882311F081E01DC016FF08C056
:1094100080E062E00E945746882311F082E013C08A
:1094200015FF08C080E063E00E945746882311F0D2
:1094300083E009C014FF09C080E064E00E94574641
:10944000882319F084E08093FE0E80916A0E8823B1
:10945000B9F081E08093610E809395018091720E46
:1094600080936B0E20914F0E2F5F20934F0E8091B3
:10947000930190E030E02817390714F010924F0E56
:109480001F910895CF93DF9380919501882399F1DF
:109490000E945A428FEF8093A4098093A70980937A
:1094A000AA098093AD0986EF9CE09093060A809309
:1094B000050A8FEB97E30E9487421092510E10929B
:1094C000500E1092010F1092000F1092540E109235
:1094D000490E109295018091400E9091410E90930B
:1094E000450E8093440E8091420E9091430E9093CE
:1094F000470E8093460E1092770E24C01092E30E12
:1095000018C08091530E90E0AC01E6E0440F551F67
:10951000EA95E1F7880F991F480F591F4D505E4B90
:109520008091770E0E94003B8091E30E885F8093CC
:10953000E30E6091E30E693120F38091770E885F2E
:109540008093770E8091770E8631C0F21092770E5D
:10955000C3E1D0E02EC01092E30E22C070E090E094
:109560002091000F3091010FFC01E21BF30B6C9F67
:1095700090016D9F300D7C9F300D1124E20FF31F81
:10958000EC56FE4BE491E093ED0E1092EE0E4E2F52
:1095900050E00E942E488091E30E8F5F8093E30E8F
:1095A0006091E30E8091770E6630C0F28F5F8093FA
:1095B000770E2091000F3091010F8091770E90E08F
:1095C0008217930744F2233131053CF42F5F3F4F5C
:1095D0003093010F2093000F97C08091500E90910F
:1095E000510E01969093510E8093500E4091640E4F
:1095F000542F5E5F9091E30E81E016C09FE0865F7E
:10960000282F30E08A50E92FF0E065E0EE0FFF1FD1
:109610006A95E1F7E20FF31FE056FA4F50839F5F20
:10962000953189F78F5F97E08A3040F39093E30E8E
:10963000942F9F5F81E00CC0865FE82FF0E0E0563A
:10964000FA4FE054FE4F9083E052FF4F90838950D1
:109650008A3090F381E00DC0825FE82FF0E055E0A2
:10966000EE0FFF1F5A95E1F7E056FA4F9287948B61
:109670008D50873088F38093770E842F8D5F809391
:109680006A078093740780934A0880935408E09196
:10969000540EE05FF0E035E0EE0FFF1F3A95E1F782
:1096A000E056FA4F4C5F43878CE090E060E170E059
:1096B00046E953E30E94873B8CE090E061E170E073
:1096C0004FE953E30E94873B8CE090E062E170E059
:1096D00048EA53E30E94873B8CE090E063E170E04E
:1096E00041EB53E30E94873B84E090E069E170E046
:1096F0004AEB53E30E94873B82E190E066E070E032
:109700004FEC53E30E94873B8091500E9091510E95
:10971000813F910570F091E09093950182E08093F4
:10972000490E1092610E90939A0181E090E00E94A0
:109730006C3B2091400E3091410E30FF48C080912B
:10974000440E9091450E90FD42C084E06FEF41E0E1
:109750000E94F8328091500E9091510E0E94B45A9E
:109760008091540E8130C9F0813030F08230D9F0D0
:10977000833009F05AC01BC082E08093610E80E004
:1097800091E09093470E8093460E9093450E809300
:10979000440E81E0809395014CC084E06FEF41E07E
:1097A0000E94F83242C084E08093610E42C08093F0
:1097B000490E1092610E1092540E81E080939A012E
:1097C00080935F0E80935E0E81E090E030C027FFB3
:1097D00014C08091440E87FD10C085E06FEF41E01A
:1097E0000E94F8328091540E81508093540E843040
:1097F000C0F083E08093540E14C026FF16C0809101
:10980000440E86FD12C085E06FEF41E00E94F83201
:109810008091540E8F5F8093540E843010F010921C
:10982000540E1092510E1092500E82E090E00E9461
:109830006C3BDF91CF910895EF92FF920F931F93AE
:10984000CF93DF9380919A018823D1F11092A209DE
:109850008FEF8093A4098093A7098093AA0980932E
:10986000AD0910929A0106EF1CE0C8010E948742E0
:109870001093060A0093050A1092770E02E41CC0AA
:109880001092E30E10C04091650E409FA00111247C
:109890004D505E4B8091770E0E94003B8091E30E0D
:1098A000885F8093E30E6091E30E693160F38091ED
:1098B000770E885F8093770E8091770E863100F364
:1098C0008FEF8093A4098093A7098093AA098093BE
:1098D000AD098091590E882309F06CC00E94F143B4
:1098E000809199018093A5094091F70E50E08091F5
:1098F000EF0E06E0809FC00111242091F90E3091F7
:10990000FA0EB901469F9001479F300D569F300DCA
:109910001124820F8A5F8093A3098091FC0E880F27
:10992000880F880F2091020F3091030FB901469FD5
:109930009001479F300D569F300D1124820F885F94
:109940008093A409809194018230A1F581E00E9466
:10995000F143809199018093A8094091F80E50E05D
:109960008091F00E809FC00111242091F90E30915A
:10997000FA0EB901469F9001479F300D569F300D5A
:109980001124820F8A5F8093A6098091FD0E880FB3
:10999000880F880F2091020F3091030FB901469F65
:1099A0009001479F300D569F300D1124820F885F24
:1099B0008093A7091092E40E05E110E0E6E0EE2E98
:1099C000FF24F394FDC01092F40EF0C010926D0EBF
:1099D00090E0809FF001819FF00D909FF00D112489
:1099E000E20FF11DE356FE4F808190E09093E00E70
:1099F0008093DF0E892B09F4D4C01092770EB2C089
:109A0000A32FB0E0FD01EF50F14F20818091E40ED3
:109A1000281709F0A2C0AB50B14FEC918091F40E21
:109A2000E81709F09AC08091DF0E9091E00EF0E007
:109A3000422F50E02091640E049759F475E0EE0F28
:109A4000FF1F7A95E1F7E40FF51FE056FA4F2E5FFE
:109A50000AC065E0EE0FFF1F6A95E1F7E40FF51FFE
:109A6000E056FA4F2D5F2083832F0E94F1438091AF
:109A7000770EA82FB0E0AD014E5F5F4F6091F90EF9
:109A80007091FA0EFD01E950F14F8081C82FD0E0AE
:109A9000FD01EF50F14F80818E9DC0011124C69FC2
:109AA0009001C79F300DD69F300D1124820F8A5F21
:109AB000FA01EE0FFF1FE40FF51FE056F64F80830B
:109AC0009B0177FF04C022273327261B370B243046
:109AD00031054CF0FA01EE0FFF1FE40FF51FE056C1
:109AE000F64F860F80836091020F7091030FAB5089
:109AF000B14F2C91220F220F220FC69FC001C79F8A
:109B0000900DD69F900D1124280F285FFA01EE0FBB
:109B1000FF1FE40FF51FE056F64F2183CB0177FFBF
:109B200004C088279927861B970B07974CF0FA01EA
:109B3000EE0FFF1FE40FF51FE056F64F260F2183AF
:109B4000FA01EE0FFF1FE40FF51FE056F64F80916C
:109B5000640E8C5F8283F0926D0E8091770E8F5F22
:109B60008093770E3091770E80919401381708F426
:109B700047CF80916D0E8823A1F4E091F40EF0E0C0
:109B80008091E40EA5E0EE0FFF1FAA95E1F7E80F24
:109B9000F11DE056FA4F8091DF0E9091640E890F0F
:109BA00080838091F40E8F5F8093F40E8091F40E89
:109BB0002091E40E843108F409CF2F5F2093E40E46
:109BC0008091E40E843108F4FECE8091490E8230FB
:109BD00009F052C08091500E9091510E01969093D1
:109BE000510E8093500E459738F088E090E069E17F
:109BF00070E044E40E94833B8091500E9091510E9E
:109C0000899738F089E090E069E170E045E40E94CE
:109C1000833B8091500E9091510ECD9738F08AE0A1
:109C200090E069E170E04DE40E94833B8091500E2A
:109C30009091510E8135910538F08BE090E069E10B
:109C400070E04FE40E94833B8091500E9091510E42
:109C50008937910590F14091650E82E4489FA001FB
:109C600011244D505E4B88E068E10E94003B109249
:109C7000510E1092500E21C08330F9F480E090E034
:109C800069E170E04AED53E30E94873B8091640EE6
:109C900090919601890F8093C5088BE090E069E16F
:109CA00070E0409197010E94A33B8EE090E069E153
:109CB00070E0409198010E94A33B81E090E00E94F7
:109CC0006C3BDF91CF911F910F91FF90EF90089522
:109CD0001F9380915E0E882309F446C09091F30E85
:109CE000943120F08091FB0E843130F49093EF0E8C
:109CF0008091FB0E8093FC0E10925E0E1092480E27
:109D000011E010935F0E10939A010E941C4C0E9468
:109D1000AF2F89E996E40E94672F1093710E10927D
:109D20006C0E1092770E17C01092E30E0BC080914C
:109D3000770E4BEF52E40E94003B8091E30E885F68
:109D40008093E30E6091E30E693188F38091770E82
:109D5000885F8093770E8091770E863128F30E947A
:109D600091480E941C4C8AC22091500E3091510E95
:109D70002F5F3F4F3093510E2093500EC90163E087
:109D800070E00E94CB5AE091980150919701409168
:109D9000640E892B71F0F0E085E0EE0FFF1F8A95CD
:109DA000E1F7E50FF11DE056FA4F80919601480F5B
:109DB0000AC0F0E015E0EE0FFF1F1A95E1F7E50F7E
:109DC000F11DE056FA4F40832F3F310520F01092ED
:109DD000510E1092500E8091590E882309F43FC203
:109DE0009FEF9093A4099093A7099093AA09909349
:109DF000AD0980915C0E882309F480C08091540ED7
:109E0000823010F01092540E8091640E382F3E5F15
:109E10002091E30E91E016C027E09D5F492F50E0AE
:109E20009350E22FF0E0B5E0EE0FFF1FBA95E1F797
:109E3000E40FF51FE056FA4F30832F5F2D3089F77E
:109E40009F5F27E09F3040F32093E30E282F2F5F82
:109E500091E00CC09D5FE92FF0E0E056FA4FE0542E
:109E6000FF4F2083E052FF4F208392509F3090F3AA
:109E700091E00DC09A5FE92FF0E0A5E0EE0FFF1F23
:109E8000AA95E1F7E056FA4F2383228B955097303D
:109E900088F39093770E8D5F8093630680937206AC
:109EA000809343078093520784E090E067E070E07E
:109EB00049EA57E30E94873B85E090E069E070E063
:109EC00047EB57E30E94873B85E090E06AE070E053
:109ED0004BEB57E30E94873B8091640E809388068A
:109EE000E091540EE75FF0E075E0EE0FFF1F7A950A
:109EF000E1F7E056FA4F8C5F8483B1C18091600E28
:109F00002091E30E4091640E882309F413C19093CD
:109F1000A4099093A7099093AA099093AD09542F8F
:109F20005E5F922F81E012C0F0E065E0EE0FFF1F50
:109F30006A95E1F7E20FF31FE056FA4F5083E92FDD
:109F40009E2F9F5F9A3181F78F5F99E1853120F4D1
:109F5000E1E0282F30E0F4CF9093E30E942F9F5F41
:109F600081E009C0E82FF0E0E056FA4F9083E05E10
:109F7000FC4F90838F5F8531A8F381E00CC0E82F00
:109F8000F0E025E0EE0FFF1F2A95E1F7E056FA4FCB
:109F90009083958B8F5F893190F38093770E842F18
:109FA0008D5F8093A0058093B5058093C008809352
:109FB000D50881E090E061E070E043E354E30E9463
:109FC000873B81E090E062E070E048E454E30E9467
:109FD000873B81E090E063E070E04DE554E30E9450
:109FE000873B81E090E064E070E04DE554E30E943F
:109FF000873B81E090E065E070E042E754E30E9437
:10A00000873B81E090E066E070E047E854E30E941F
:10A01000873B81E090E067E070E04CE954E30E9408
:10A02000873B81E090E068E070E041EB54E30E9400
:10A03000873B81E090E069E070E04DE554E30E94E9
:10A04000873B81E090E06AE070E04DE554E30E94D8
:10A05000873B81E090E06BE070E046EC54E30E94C7
:10A06000873B81E090E06CE070E04BED54E30E94B0
:10A07000873B81E090E06DE070E04DE554E30E94A5
:10A08000873B81E090E06EE070E04DE554E30E9494
:10A09000873B81E090E06FE070E040EF54E30E9486
:10A0A000873B81E090E060E170E045E055E30E948D
:10A0B000873B81E090E061E170E04AE155E30E9476
:10A0C000873B81E090E062E170E04FE255E30E945F
:10A0D000873B81E090E063E170E044E455E30E9457
:10A0E000873B81E090E064E170E049E555E30E9440
:10A0F000873B81E090E065E170E04DE554E30E942C
:10A10000873B81E090E066E170E04DE554E30E941A
:10A11000873B81E090E067E170E04EE655E30E9406
:10A12000873B81E090E068E170E043E855E30E94FE
:10A13000873BA4C09093A4099093A7099093AA0980
:10A140009093AD09542F5E5F922F81E016C097E087
:10A150008B5F282F30E08550E92FF0E015E0EE0FFF
:10A16000FF1F1A95E1F7E20FF31FE056FA4F5083F5
:10A170009F5F9F3089F78F5F99E08D3040F3909318
:10A18000E30E942F9F5F81E00CC08B5FE82FF0E01F
:10A19000E056FA4FE054FF4F9083E05EFE4F90830D
:10A1A00084508D3090F381E00DC08A5FE82FF0E09D
:10A1B000B5E0EE0FFF1FBA95E1F7E056FA4F958331
:10A1C000928B8550893088F38093770E842F8D5F32
:10A1D000809365068093720680938507809392072B
:10A1E00087E090E068E070E04BEE53E30E94873B2D
:10A1F00087E090E069E070E047EF53E30E94873B1F
:10A2000087E090E06AE070E043E054E30E94873B1F
:10A2100087E090E06BE070E04FE054E30E94873B02
:10A2200087E090E06CE070E047E254E30E94873BF7
:10A2300087E090E06DE070E04BE154E30E94873BE3
:10A24000E091540EE85FF0E0A5E0EE0FFF1FAA9545
:10A25000E1F7E056FA4F8091640E8C5F868380911F
:10A260005F0E882321F480919A01882339F00E949F
:10A270001C4C10925F0E10929A0104C081E090E095
:10A280000E946C3B1F9108958091FE0E8823B9F4C3
:10A290000E940446882399F08091580E882331F05B
:10A2A00083E08093490E0E949148089580916B0E3F
:10A2B0008F5F80936B0E82E08093610E0895809192
:10A2C000490E833019F40E94684E08950E94EA46B0
:10A2D00008951F9311E01093580E10939A01109354
:10A2E0005F0E0E945A420E941C4C81E090E00E9446
:10A2F0006C3B1092490E1092610E1093710E0E94E9
:10A300005A4210939A010E941C4C1F91089580910B
:10A31000590E882309F490C02091400E3091410ECF
:10A3200027FF0FC08091440E87FD0BC08091540E13
:10A3300081508093540E8F3F99F485E08093540EA2
:10A340000FC026FF0DC08091440E86FD09C080918C
:10A35000540E8F5F8093540E863010F01092540E7E
:10A3600030FF0BC12091440E3091450E30FD05C1E8
:10A3700080915C0E882379F08091540E882309F433
:10A3800057C0813009F0F9C010925C0E8093590ECD
:10A390001092540E08958091600E882339F0109227
:10A3A000600E3093410E2093400E08958091540E1C
:10A3B000823011F1833030F4882361F0813009F06C
:10A3C000DCC015C0843021F18430F8F0853009F00C
:10A3D000D4C022C082E080935D0E81E08093490E5C
:10A3E0008093580E1092590E0E946951089580E092
:10A3F0000E94714881E004C081E00E94714884E0BD
:10A400006FEF41E00E94F83208951092590E0895BE
:10A4100081E08093600E089580915A0E882341F068
:10A4200080915B0E882321F481E080935C0E089577
:10A4300080E00E947B4808952091400E3091410EAB
:10A4400027FF0AC08091440E87FD06C080919801C5
:10A45000882311F081500BC026FF11C08091440E5B
:10A4600086FD0DC080919801833148F48F5F809301
:10A47000980181E080939A0180935F0E53C025FF7D
:10A480000AC08091440E85FD06C080919701882303
:10A4900011F081500BC024FF0CC08091440E84FD4C
:10A4A00008C080919701833120F48F5F80939701DA
:10A4B000E0CF22FF0EC08091440E82FD0AC0809141
:10A4C0009701833130F480919601873010F48F5FCB
:10A4D00011C032FF12C08091440E9091450E92FD42
:10A4E0000CC080919701833140F4809196018823BC
:10A4F00021F0815080939601BCCF30FF13C0809132
:10A50000440E9091450E90FD0DC081E08093590E50
:10A5100080939A0110925F0E0E941C4C81E090E0A3
:10A520000E946C3B8091400E9091410E93FF25C09C
:10A53000609197015091980140919601252F30E04C
:10A5400085E190E0289FF001299FF00D389FF00DE4
:10A550001124E60FF11DE356FE4F408381E0809306
:10A560005A0E80935F0E463040F06093EF0E50938A
:10A57000FC0E6093F30E5093FB0E08951F93182F5B
:10A580000E94DC44812F0E9498440E94464481E04E
:10A5900080939A010E941C4C1F9108951F938091F3
:10A5A00095018823E1F0109295011092540E80914C
:10A5B0006B0E8F5F809356038FEF8093A409809377
:10A5C000A7098093AA098093AD0980E091E0909358
:10A5D000450E8093440E9093410E8093400E40911F
:10A5E000640E542F5E5F9091E30E81E016C099E0F7
:10A5F0008D5F282F30E08350E92FF0E065E0EE0F0B
:10A60000FF1F6A95E1F7E20FF31FE056FA4F508300
:10A610009F5F923189F78F5F9AE08F3040F390937C
:10A62000E30E942F9F5F81E00CC08D5FE82FF0E078
:10A63000E056FA4FE050FF4F9083E05CFE4F90836E
:10A6400082508F3090F381E00DC0885FE82FF0E0FA
:10A6500025E0EE0FFF1F2A95E1F7E056FA4F9383AE
:10A66000928B87508A3088F38093770E842F8D5F8A
:10A670008093A3068093B2068093E3078093F2074A
:10A68000E091540EE65FF0E095E0EE0FFF1F9A9523
:10A69000E1F7E056FA4F4C5F448385E090E06AE0D2
:10A6A00070E043E457E30E94873B80E190E06AE07A
:10A6B00070E0409156030E94A33B85E090E06BE080
:10A6C00070E041E557E30E94873B84E58093A3094E
:10A6D00080E68093A409809199018093A50985E083
:10A6E00090E06CE070E04FE557E30E94873B85E027
:10A6F00090E06DE070E04DE657E30E94873B4091AB
:10A700009B01442339F08CE090E06DE070E00E9402
:10A71000A33B08C08CE090E06DE070E045EA57E3B1
:10A720000E94873B85E090E06EE070E04BE757E3E6
:10A730000E94873B85E090E06FE070E049E857E3D6
:10A740000E94873B85E090E060E170E047E957E3D5
:10A750000E94873B8091400E9091410E90FF62C015
:10A760008091440E9091450E90FD5CC08091540EF6
:10A770008430B9F1853030F4882351F0833009F00A
:10A7800051C020C08530A1F1863009F04BC042C0D5
:10A790004091560320916B0E30E0842F90E001979A
:10A7A0002817390709F43CC1415040936B0E82E0F1
:10A7B0008093610E81E08093950180939A010E94BD
:10A7C0001C4C2AC180919B01882361F10E94AF2F0C
:10A7D00089E996E40E94672F80EB97E40E94812F1D
:10A7E00021C082E08093610E81E08093950118C1C1
:10A7F0001092610E81E08093950180939A0180E030
:10A8000091E09093450E8093440E9093410E809377
:10A81000400E06C181E08093610E809395011092F5
:10A82000490EFEC09091400E97FF15C08091440ED6
:10A8300087FD11C085E06FEF41E00E94F832809102
:10A84000540E81508093540E8F3F09F0CAC086E0A9
:10A850008093540EC6C096FF14C08091440E86FDAE
:10A8600010C085E06FEF41E00E94F8328091540EF5
:10A870008F5F8093540E873008F4B3C01092540E4B
:10A88000B0C095FF53C08091440E85FD4FC010911C
:10A89000540E113099F0113030F0123001F11330B4
:10A8A00009F09FC02CC084E06FEF41E00E94F832B5
:10A8B0008091560381508093560393C084E06FEFDC
:10A8C00041E00E94F8328091620E81508093620EC6
:10A8D0008F3F09F086C082E08093620E82C084E0E0
:10A8E0006FEF41E00E94F8328091630E81508093B7
:10A8F000630E8F3F09F075C01093630E72C084E041
:10A900006FEF41E00E94F83280919B01815080936B
:10A910009B0181508E3F08F45AC010929B010E9407
:10A92000AF2F89E996E40E94672F5BC094FF59C05E
:10A930008091440E84FD55C08091540E8130C9F041
:10A94000813030F0823021F1833009F04AC02FC0CD
:10A9500084E06FEF41E00E94F832809156038F5FF0
:10A9600080935603909192019817D8F590935603CF
:10A9700038C084E06FEF41E00E94F8328091620EAF
:10A980008F5F8093620E833060F11092620E29C057
:10A9900084E06FEF41E00E94F8328091630E8F5F98
:10A9A0008093630E8330E8F01092630E1AC084E047
:10A9B0006FEF41E00E94F83280919B018F5F80939E
:10A9C0009B0190919C01981710F490939B010E9419
:10A9D000AF2F89E996E40E94672F80EB97E40E94ED
:10A9E000812F9091620E992311F486E005C086E0D4
:10A9F000989FC00111248F53809399019091630E09
:10AA0000992319F41092640E07C086E0989FC00144
:10AA1000112485548093640E81E090E00E946C3B89
:10AA20001F91089580919501882369F01092540E2A
:10AA3000109295018FEF8093A4098093A7098093CA
:10AA4000AA098093AD098091550E882309F424C189
:10AA50008091400E9091410E90FF08C08091440E6D
:10AA60009091450E90FD02C01092550E8FEF80938D
:10AA7000A4098093A7098093AA098093AD098091C6
:10AA8000640E582F5E5F2091E30E91E012C0F0E05B
:10AA9000B5E0EE0FFF1FBA95E1F7E20FF31FE056A6
:10AAA000FA4F5083E42F4E2F4F5F4A3181F79F5F5B
:10AAB00029E1953120F4E1E0292F30E0F4CF209313
:10AAC000E30E282F2F5F91E009C0E92FF0E0E05658
:10AAD000FA4F2083E05EFC4F20839F5F9531A8F3FF
:10AAE00091E00CC0E92FF0E0A5E0EE0FFF1FAA9562
:10AAF000E1F7E056FA4F2083258B9F5F993190F361
:10AB00009093770E8D5F8093A0058093B505809319
:10AB1000C0088093D50881E090E061E070E04DEAE4
:10AB200055E30E94873B81E090E062E070E04DE5F4
:10AB300054E30E94873B81E090E063E070E04DE5E4
:10AB400054E30E94873B81E090E064E070E042ECD7
:10AB500055E30E94873B81E090E065E070E047EDBF
:10AB600055E30E94873B81E090E066E070E04CEEA8
:10AB700055E30E94873B81E090E067E070E041E0B0
:10AB800056E30E94873B81E090E068E070E046E198
:10AB900056E30E94873B81E090E069E070E04BE281
:10ABA00056E30E94873B81E090E06AE070E040E479
:10ABB00056E30E94873B81E090E06BE070E04DE55A
:10ABC00054E30E94873B81E090E06CE070E04DE54B
:10ABD00054E30E94873B81E090E06DE070E045E542
:10ABE00056E30E94873B81E090E06EE070E04AE629
:10ABF00056E30E94873B81E090E06FE070E04FE712
:10AC000056E30E94873B81E090E060E170E04DE513
:10AC100054E30E94873B81E090E061E170E04DE504
:10AC200054E30E94873B81E090E062E170E044E9F8
:10AC300056E30E94873B81E090E063E170E049EADF
:10AC400056E30E94873B81E090E064E170E04EEBC8
:10AC500056E30E94873B81E090E065E170E04DE5BE
:10AC600054E30E94873B81E090E066E170E04DE5AF
:10AC700054E30E94873B81E090E067E170E043EDA0
:10AC800056E30E94873B81E090E068E170E048EE87
:10AC900056E30E94873B38C21092770E24C0109270
:10ACA000E30E18C08091530E90E0AC01E6E0440F33
:10ACB000551FEA95E1F7880F991F480F591F4D500E
:10ACC0005E4B8091770E0E94003B8091E30E885F7F
:10ACD0008093E30E6091E30E693120F38091770E4B
:10ACE000885F8093770E8091770E8631C0F2409115
:10ACF000640E642F6E5F2091E30E81E016C09FE02A
:10AD00008B5F282F30E08550E92FF0E055E0EE0F03
:10AD1000FF1F5A95E1F7E20FF31FE056FA4F6083E9
:10AD20009F5F973189F78F5F29E08B3040F3942F35
:10AD30009F5F81E00CC08B5FE82FF0E0E056FA4F98
:10AD4000E054FE4F9083E05EFE4F908384508B3042
:10AD500090F381E00DC0825FE82FF0E035E0EE0F68
:10AD6000FF1F3A95E1F7E056FA4F9583908B8D508F
:10AD7000893088F3542F5D5F5093650750937007B7
:10AD8000509385085093900880E00CC08B5FE82FAB
:10AD9000F0E0E056FA4FE05AFF4F9083E054FF4F47
:10ADA000908384508A3090F380E00DC08D5FE82F4F
:10ADB000F0E0B5E0EE0FFF1FBA95E1F7E056FA4F6D
:10ADC000958396878250863088F381E016C094E0A0
:10ADD0008B5F282F30E08550E92FF0E0A5E0EE0FE3
:10ADE000FF1FAA95E1F7E20FF31FE056FA4F6083C9
:10ADF0009F5F993089F78F5F26E0893040F3209379
:10AE0000E30E8093770E509368064C5F409369067B
:10AE10004F5F40936B0686EF9CE00E9487428AE278
:10AE20008093A30988E38093A4098091990180937A
:10AE3000A509E091540EE05FF0E075E0EE0FFF1F12
:10AE40007A95E1F7E056FA4F8091640E8C5F868325
:10AE500087E090E06DE070E04DEF56E30E94873BA5
:10AE600087E090E060E170E047E057E30E94873BB5
:10AE700087E090E061E170E041E157E30E94873BA9
:10AE800087E090E062E170E04BE157E30E94873B8E
:10AE900040916B0E4F5F8DE090E062E170E00E94A8
:10AEA000A33B87E090E063E170E045E257E30E9456
:10AEB000873B87E090E064E170E049E357E30E945C
:10AEC000873B40919B01442339F08DE090E064E1A1
:10AED00070E00E94A33B08C08DE090E064E170E068
:10AEE00045EA57E30E94873B87E090E065E170E028
:10AEF0004FE257E30E94873B2091400E3091410E74
:10AF000030FF20C08091440E9091450E90FD1AC0F4
:10AF10008091540E853079F481E06FEF41E00E941A
:10AF2000F8321092490E81E08093610E8093950172
:10AF300082E090E0EBC0833009F0CBC081E08093E9
:10AF4000550E089527FF15C08091440E87FD11C04E
:10AF500085E06FEF41E00E94F8328091540E8150FD
:10AF60008093540E8F3F09F0B4C085E08093540E57
:10AF7000B0C026FF14C08091440E86FD10C085E04D
:10AF80006FEF41E00E94F8328091540E8F5F809302
:10AF9000540E863008F49DC01092540E9AC025FFBE
:10AFA0004AC08091440E85FD46C08091540E813088
:10AFB000A1F0813030F08230E1F0843009F089C0B6
:10AFC00026C08091630E81508093630E8F3F09F0FD
:10AFD00065C082E08093630E61C08091620E8150F3
:10AFE0008093620E8F3F09F059C082E08093620E19
:10AFF00055C080916B0E815080936B0E8F3F09F08E
:10B000004DC080919201815080936B0E47C080911A
:10B010009B01815080939B0181508E3F08F459C061
:10B0200010929B0180EB97E40E94AF2F89E996E490
:10B030000E94672F4EC024FF4CC08091440E84FDB7
:10B0400048C08091540E813089F0813028F08230E0
:10B05000B9F08430F1F528C08091630E8F5F809342
:10B06000630E8330D8F01092630E18C08091620E88
:10B070008F5F8093620E833088F01092620E0EC054
:10B0800020916B0E2F5F20936B0E8091920190E0C8
:10B0900030E02817390714F010926B0E84E06FEF40
:10B0A00041E00E94F83215C080919B018F5F809330
:10B0B0009B0190919C01981710F490939B010E9422
:10B0C000AF2F89E996E40E94672F80EB97E40E94F6
:10B0D000812F9091620E992311F486E005C086E0DD
:10B0E000989FC00111248F53809399019091630E12
:10B0F000992319F41092640E07C086E0989FC0014E
:10B10000112485548093640E81E090E00E946C3B92
:10B1100008950F931F9380919501882309F449C0E6
:10B120000E945A428FEF8093A4098093A7098093CD
:10B13000AA098093AD0986EF9CE09093060A80935C
:10B14000050A1092510E1092500E1092950181E056
:10B1500080939A011092770E28C01092E30E1CC0C3
:10B160000E94AF5A64E070E00E94DF5A9C01AC017B
:10B1700096E0440F551F9A95E1F7220F331F420FB7
:10B18000531F4D505E4B812F602F0E94003B8091DA
:10B19000E30E885F8093E30E0091E30E1091770E2B
:10B1A0000931F0F2185F1093770E8091770E863197
:10B1B000A0F288E090E06AE070E049EC53E30E947E
:10B1C000873B40916B0E4F5F8EE090E06AE070E04D
:10B1D0000E94A33B81E0809395011092610E8093C1
:10B1E000490E0E9491488EE190E00E946C3B1F91B5
:10B1F0000F9108952091610E222349F18091520E02
:10B200008F5F8093520E8F3140F08091530E91E00A
:10B2100089278093530E1092520E81E08093480E3E
:10B22000223069F0233018F4213089F405C024302D
:10B2300049F0253061F409C00E94424A08950E94F5
:10B24000895808950E94125508950E94CE5208957B
:10B25000FF920F931F93CF93DF930E944748B5E06F
:10B26000FB2E1092770E19C0E22FF0E0EE0FFF1FB9
:10B270008F01005C114FD8018D919C91EC5BF14FD7
:10B2800091838083822F0E945243F80191838083AF
:10B290008091770E8F5F8093770E2091770E80914B
:10B2A0009401281708F32091490E223019F40E94C6
:10B2B0006D49F1C0233019F40E948751ECC0809190
:10B2C000610E882309F0E7C0213089F48091400E97
:10B2D0009091410E90FF0BC08091440E9091450ECD
:10B2E00090FD05C0F092610E20939501D4C010929C
:10B2F000770ECAC0CE2FD0E0DE01AA0FBB1FFD0122
:10B30000E05CF14F2081318130FF12C0AC5BB14F66
:10B310008D919C9190FD0CC08091490E823041F43A
:10B320001092490E81E08093610E8093480EB3C065
:10B33000FE01E250F14F8081882309F0A0C031FF67
:10B3400014C0CC0FDD1FCC5BD14F8881998191FD5A
:10B350000CC08091580E882331F083E08093490E11
:10B360000E94914898C00E9491488091770EC82F02
:10B37000D0E0DE01AA0FBB1FFD01E05CF14F0190A0
:10B38000F081E02DE2FF07C0AC5BB14F8C9182FDF4
:10B3900002C081E00BC0F2FF0BC0CC0FDD1FCC5B05
:10B3A000D14F8881998192FD03C080E00E94BE52F6
:10B3B0009091770EA92FB0E0FD01E250F14F80810E
:10B3C000882309F05CC0AA0FBB1FA05CB14F8C9111
:10B3D00087FF0DC0892F61E00E945746882339F00E
:10B3E000E091770EF0E0E250F14F81E047C090919C
:10B3F000770EE92FF0E0EE0FFF1FE05CF14F808148
:10B4000086FF0DC0892F62E00E945746882339F0DD
:10B41000E091770EF0E0E250F14F82E02FC0909182
:10B42000770EE92FF0E0EE0FFF1FE05CF14F808117
:10B4300085FF0DC0892F63E00E945746882339F0AD
:10B44000E091770EF0E0E250F14F83E017C0909169
:10B45000770EE92FF0E0EE0FFF1FE05CF14F8081E7
:10B4600084FF0DC0892F64E00E945746882339F07D
:10B47000E091770EF0E0E250F14F84E0808380911C
:10B48000770E8F5F8093770EE091770E8091940115
:10B49000E81708F42FCF8091610E882319F00E94DD
:10B4A000FA58DFCE8091490E833019F40E94684E1D
:10B4B000D8CE0E9444510E941C4CD3CEA0E0B0E0F4
:10B4C000E4E6FAE50C94565BEC01A880B980CA80EA
:10B4D000DB80A114B104C104D10441F484E2A82E9C
:10B4E00089EDB82E8BE5C82E87E0D82EC601B501B0
:10B4F0002DE133EF41E050E00E94335B27EA31E475
:10B5000040E050E00E94145B7B018C01C601B50154
:10B510002DE133EF41E050E00E94335BCA01B901F5
:10B520002CEE34EF4FEF5FEF0E94145B6E0D7F1D2A
:10B53000801F911F97FF04C0615070408040904869
:10B54000688379838A839B839B013F77C901CDB749
:10B55000DEB7EAE00C94725B0E945E5A089587E5BC
:10B5600093E00E945E5A0895A0E0B0E080935703F4
:10B5700090935803A0935903B0935A030895991BCD
:10B5800079E004C0991F961708F0961B881F7A95DA
:10B59000C9F780950895AA1BBB1B51E107C0AA1FDC
:10B5A000BB1FA617B70710F0A61BB70B881F991F64
:10B5B0005A95A9F780959095BC01CD01089597FB08
:10B5C000092E07260AD077FD04D0E5DF06D000203B
:10B5D0001AF4709561957F4F0895F6F790958195CF
:10B5E0009F4F0895A1E21A2EAA1BBB1BFD010DC09F
:10B5F000AA1FBB1FEE1FFF1FA217B307E407F50723
:10B6000020F0A21BB30BE40BF50B661F771F881FFE
:10B61000991F1A9469F760957095809590959B0194
:10B62000AC01BD01CF010895629FD001739FF0016D
:10B63000829FE00DF11D649FE00DF11D929FF00DC2
:10B64000839FF00D749FF00D659FF00D9927729FF9
:10B65000B00DE11DF91F639FB00DE11DF91FBD0184
:10B66000CF011124089597FB092E05260ED057FD12
:10B6700004D0B8DF0AD0001C38F4509540953095BE
:10B6800021953F4F4F4F5F4F0895F6F79095809566
:10B69000709561957F4F8F4F9F4F08952F923F92E6
:10B6A0004F925F926F927F928F929F92AF92BF92D2
:10B6B000CF92DF92EF92FF920F931F93CF93DF937E
:10B6C000CDB7DEB7CA1BDB0B0FB6F894DEBF0FBEDB
:10B6D000CDBF09942A88398848885F846E847D8428
:10B6E0008C849B84AA84B984C884DF80EE80FD802A
:10B6F0000C811B81AA81B981CE0FD11D0FB6F894A0
:0EB70000DEBF0FBECDBFED010895F894FFCF60
:10B70E00000000000000000000000000000000002B
:10B71E00000000000000000000000000000000001B
:10B72E00000000000000000000000000000000000B
:10B73E0000000000000000000000000000000000FB
:10B74E0000000000000000000000000000000000EB
:10B75E0000000000000000000000000000000000DB
:10B76E0000000000000000000000000000000000CB
:10B77E0000000000000000000000000000000000BB
:10B78E0000000000000000000000000000000000AB
:10B79E00D03D06030101010C02060101010000006B
:10B7AE00000000000000000000000000000000008B
:10B7BE00000100000001010101010101010101016F
:10B7CE00010000000000010000000102020202025E
:10B7DE00020202020201000000000001000000014E
:10B7EE00020202020602020304020100000000002F
:10B7FE000100000001010101020202020202020127
:10B80E000000000000010000000000000102020222
:10B81E000202020201000000000001000000000010
:10B82E0000010202020202020201000000000001F9
:10B83E0000000000000001020202020202020100EA
:10B84E0000000000010000000000000102020202E0
:10B85E0002020201000000000001000000000000D2
:10B86E0001020202020202020100000000000100B9
:10B87E0000000000000101010101010101010000B1
:10B88E0000000001000000000000000000000000A9
:10B89E000000000000000000010000000000000099
:10B8AE000000000000000000000000000001000089
:10B8BE00000000000000000000000000000000007A
:10B8CE000000010000000000000000000000000069
:10B8DE000000000000000001000000000000000059
:10B8EE000000000000000000000000000100000049
:10B8FE00000000000000000000000000000000003A
:10B90E000001000000000000000000000000000028
:10B91E000000000000000100000000000000000018
:10B92E000000000000000000000000010000000008
:10B93E0000000000000000000000000000000000F9
:10B94E0001000000000000000000000000000000E8
:0CB95E00000000000000010100000000DB
:00000001FF
